:020000040040BA
:10400000B84B002021A740001DA740001DA740007D
:104010001DA740001DA740001DA740000000000094
:10402000000000000000000000000000C1AA4000E5
:104030001DA740000000000021AB400085AB400000
:104040001DA740001DA740001DA740001DA7400060
:104050001DA740001DA740001DA740000000000054
:104060001DA740003DC340000000000085834000C4
:10407000998340002D9F40001DA740001DA74000D0
:104080001DA740001DA740003D9F400095634000D4
:1040900051C340001DA740001DA74000ED4C40004B
:1040A0001DA740001DA740001DA740001DA7400000
:1040B0001DA74000D14B40001DA74000000000009C
:1040C00000000000000000000000000000000000F0
:1040D00000000000000000000000000000000000E0
:1040E00000000000000000000000000000000000D0
:1040F0000000000000000000000000001DA74000BC
:10410000999440001DA7400000000000000000003E
:10411000000000000000000000000000000000009F
:10412000000000000000000000000000000000008F
:10413000000000000000000000000000000000007F
:10414000000000000000000000000000000000006F
:104400005CD2000010B5054C237833B9044B13B1CE
:104410000448AFF300800123237010BDB80B0020C7
:1044200000000000900641000C4B43B10C480D49C0
:1044300010B5AFF300800C48036823B910BD0A48DB
:10444000036833B97047094B002BF7D0BDE8104023
:104450001847064B002BF5D0184700BF000000009E
:1044600090064100BC0B00209006410000000000B7
:1044700030B587B01D20184B9847184C236C23F497
:10448000001323646846164B984769462046154B2F
:104490009847042323610823236101232361626871
:1044A00022F08F026260104A032120460F4DA84778
:1044B000002120460E4B9847636813F0800F01D10E
:1044C000082222600B4B4FF000521A60702283F8D2
:1044D0001D2307B030BD00BF65A44000008003402D
:1044E000BD4A4000514B400019454000A14B4000DF
:1044F000E54A400000E100E00222014B1A607047EB
:1045000000800340024B1880024B1980704700BFA7
:10451000820000208400002010B5064C206D80B27F
:10452000054B9847A06DE16D89B280B2034B984767
:1045300010BD00BF00800340096B400005454000EE
:10454000014B1888704700BF82000020014B18887B
:10455000704700BF840000200D4B1B8840F6896225
:10456000934205D90B4A12883E2A01D8032070478E
:10457000084A128840F689618A4203D93E2B01D845
:1045800004207047934201D80220704701207047F1
:104590008200002084000020012070477047012025
:1045A000704700207047704701207047014B187812
:1045B000704700BFDC0B00207047000058B908B5F9
:1045C000054B1B78012B00D008BD044B1B68002B4A
:1045D000FAD09847F8E77047E00B0020D40B002092
:1045E00008B50C4B9847C3780B4A1370012B0CD1BC
:1045F00001220A4B1A700022094B1A80094B984776
:10460000094B1B681BB1984701E0084B98470120F4
:1046100008BD00BFE17F4000DC0B0020E00B002064
:10462000DE0B002021C34000D40B00202DC340002E
:1046300008B5054B1B78012B00D008BD0022034BA9
:104640001A70034B9847F8E7DC0B0020E00B0020C2
:104650002DC3400010B582B0074B00930B460246B5
:1046600000218420054CA04718B9054A136801337E
:10467000136002B010BD00BFBD454000359B400037
:10468000D80B0020014B1860704700BFD40B0020EE
:104690002DE9F0474FF40046BF4B5E600B20BF4C46
:1046A000A0470C20A047BE4B4FF0400CC3F810C0F1
:1046B000C3F8A0C0C3F834C04FF0807EC3F810E048
:1046C000C3F8A0E0C3F834E0B64A01271761C2F886
:1046D000A070576302241461C2F8A04054631C61A7
:1046E000C3F8A0405C631F66C3F890705F655F62AB
:1046F000C3F88070196F39431967596F21F00101B0
:1047000059675F604FF480311966C3F8901059659E
:104710005962C3F88010186F08431867586F20F467
:104720008030586759601C61C3F8A0405C63042066
:104730005861C3F8A0005866C3F8900058655862E5
:10474000C3F88000196F21F004011967596F21F037
:104750000401596718211966C3F890105965596208
:10476000C3F880101D6F25F018051D675D6F25F0DB
:1047700018055D67596008251D66C3F890505D6592
:104780005D62C3F88050196F21F008011967596FF5
:1047900021F0080159675D6010211966C3F8901077
:1047A00059655962C3F88010D3F8708028F010085A
:1047B000C3F87080D3F8748028F01008C3F87480B0
:1047C00059604FF48028C3F81480C3F8A0804FF0DC
:1047D0002009C3F81490C3F8A090C3F810C0C3F820
:1047E000A0C0C3F834C0C3F810E0C3F8A0E0C3F819
:1047F00034E01761C2F8A07057631461C2F8A0409A
:1048000054634FF4007CC3F860C0C3F890C0C3F891
:1048100054C0C3F824C0C3F880C01C6F44EA0C0421
:104820001C675C6F24F400745C67C3F804C04FF429
:1048300080641C66C3F890405C655C62C3F880408D
:104840001F6F27431F675F6F27F480675F675C6098
:104850004FF4006EC3F810E0C3F8A0E0C3F834E0F2
:104860004FF400275F61C3F8A0701F66C3F8907013
:104870005F655F62C3F880701F6F27F400271F67B2
:104880005F6F27F400275F674FF480175F61C3F8FD
:10489000A0701F66C3F890705F655F62C3F8807098
:1048A0001F6F27F480171F675F6F27F480175F67FC
:1048B0004FF480575F61C3F8A0705F66C3F89070D3
:1048C0005F655F62C3F880701F6F27F480571F67B2
:1048D0005F6F27F480575F674FF400575F61C3F83D
:1048E000A0704FF480775761C2F8A0704FF48048F1
:1048F000C3F86080C3F89080C3F85080C3F8248068
:10490000C3F88080D3F870A02AF4804AC3F870A05E
:10491000D3F874A02AF4804AC3F874A0C3F81080B6
:10492000C3F8A080C3F830805E61C3F8A0604FF484
:1049300000365E61C3F8A0601066C2F89000506552
:104940005062C2F88000166F26F004061667566F94
:1049500026F00406566750601566C2F890505565FB
:104960005562C2F88050106F20F008001067506F39
:1049700020F00800506755600B4DD5F8140140F049
:104980003000C5F814015161C2F8A0105166C2F898
:1049900090105165516209E050140E4065A440002A
:1049A000000E0E4000100E4000020E40C2F88010B3
:1049B000116F21F010011167516F21F01001516743
:1049C000C2F81090C2F8A090C2F83490C2F810C09B
:1049D000C2F8A0C0C2F830C04FF400015961C3F85A
:1049E000A0105966C3F8901059655962C3F8801039
:1049F000196F21F400011967596F21F400015967FB
:104A0000C2F860E0C2F890E0C2F854E0C2F824E0D6
:104A1000C2F880E0116F21F400611167516F21F439
:104A200000615167C2F804E01466C2F89040546512
:104A30005462C2F88040116F21F480611167516F98
:104A400021F48061516754601F66C3F890701F6540
:104A50005F62C3F880701A6F22F480721A675A6F0F
:104A600022F480725A671F61C3F8A0701F63BDE80B
:104A7000F08700BF08B5034B53F8203003B19847C7
:104A800008BD00BFC40E002010B582B0036B0193B7
:104A9000002400E00134172C09D8064B53F82420D9
:104AA000019B1A42F6D02046034B9847F2E702B02A
:104AB00010BD00BFAC004100754A400000230360F8
:104AC000064A4260064A82604FF48022C260022297
:104AD000027442748374C374037570470000DC056C
:104AE000808D5B00036C19430164704710B58B7CAB
:104AF00023B34FF000434A688C686400B2FBF4F2C1
:104B0000013A120292B213430A7C120602F070625A
:104B100013434A7C120702F040521343CA681343FE
:104B20004360CB7C63B14FF080730A7D52B90022A1
:104B3000134303640968054B984710BD0023DAE767
:104B40000023F2E74FF48012F2E700BFE54A40008D
:104B500008B5036B13F0807F01D0192008BD012335
:104B60000360064B9847002304E00021044A42F802
:104B700023100133172BF8D9002008BDED4A40005F
:104B8000C40E0020B1F1FF3F04D0044B53F8213094
:104B9000436270474FF0FF3343627047AC004100FF
:104BA00010B5084C44F82120074A4FF00054C2F8D1
:104BB00080411B01DBB282F81D331460034B984720
:104BC00010BD00BFC40E002000E100E0854B400096
:104BD00008B50248024B984708BD00BF008003405B
:104BE000894A400010B51720234CA0471820A04741
:104BF000224B4FF480321A66C3F890205A655A62ED
:104C0000C3F88020196F11431967596F21F480315F
:104C100059675A6001225A66C3F890205A655A6251
:104C2000C3F88020196F11431967596F21F00101F2
:104C300059675A60A3F5206340F21262DA644FF4B8
:104C400000621A600E4B0F4A5A6041225A620521D7
:104C500019600D4A5A644FF4F572DA6500229A65BC
:104C600019640A4B1A700A4B4FF400021A60702242
:104C700083F8172310BD00BF65A44000000E0E404E
:104C8000000001400406090001C4000A280F0020AA
:104C900000E100E0642800D964200F4AD36D03FBD3
:104CA00000F30E49A1FB03135B09936548B10A4B5E
:104CB0005A6C22F040625A645A6C42F080625A6424
:104CC00070471346526C22F040625A645A6C42F0AC
:104CD00000625A64704700BF000001401F85EB511D
:104CE000014B1888704700BF2C0F00200F4B1B6A28
:104CF00013F0010F06D000220D490A700D490A6019
:104D00000D490A6013F0400F0ED00122084B1A70B3
:104D1000064B9A69094BB3FBF2F3064A1360C3EBE7
:104D200003139A00044B1A60704700BF0000014053
:104D3000280F0020240F00202C0F00201F1A050030
:104D4000014B1870704700BFB0000020064B1B7865
:104D500023B94FF40062054B1A6370474FF40062A9
:104D6000024B5A63704700BFB0000020000E0E4097
:104D7000064B1B7823B94FF40062054B5A6370470A
:104D80004FF40062024B1A63704700BFB00000206E
:104D9000000E0E402DE9F04186B0884616461F46AB
:104DA000D0B9244B984705460024049498238DF8E5
:104DB000043001238DF8053002238DF806300323DB
:104DC0008DF8083005AB03938DF807808DF81540FA
:104DD0002846194B984705E0184B98470546E3E7E6
:104DE0000134E4B2B4421ED28DF814403B5D8DF81C
:104DF0001630322201A92846114B9847AB79DBB215
:104E0000022BEDD028460F4B9847322201A92846A5
:104E10000B4B9847AB79DBB2022BE1D028460A4B0B
:104E20009847002003E02846074B9847012006B02A
:104E3000BDE8F08111C340000168400019C3400083
:104E40002D684000D9694000156840002DE9F04107
:104E500086B00F4616469846B8B9344B9847044674
:104E60000025049598238DF8043001238DF8053032
:104E70008DF8065002238DF8083005AB03938DF8AA
:104E8000075020462A4B98470EE02A4B9847044685
:104E9000E6E72046284B9847002044E09DF815306F
:104EA00008F805300135EDB2B54238D28DF81470EE
:104EB0008DF8155000238DF80630322201A92046C6
:104EC0001E4B9847A379DBB2022B0BD020461C4B1C
:104ED0009847322201A92046184B9847A379DBB2A4
:104EE000022BD6D101238DF80630322201A92046AB
:104EF000124B9847A379DBB2022BCFD02046104B40
:104F00009847322201A920460C4B9847A379DBB27F
:104F1000022BC3D02046084B9847002003E02046D0
:104F2000054B9847012006B0BDE8F08111C3400051
:104F30000168400019C34000156840002D6840001A
:104F4000D969400070B506460C46104BAA221A706B
:104F500011225A700222F0210D4DA847012801D0DC
:104F6000002070BD220AE4B2084B1A705C709A707F
:104F7000DC701A715C7100229A719022DA7102223F
:104F80001A720922C2213046A84770BD300F002096
:104F9000954D400010B50022054B1A7029B911211A
:104FA000034B0122034CA04710BD1021F8E700BFBE
:104FB000300F0020954D400010B50022054B1A70AF
:104FC00029B92821034B0122034CA04710BD2921F8
:104FD000F8E700BF300F0020954D400010B539B9FB
:104FE0000022044B1A7001223621034CA04710BD49
:104FF0000322F6E7300F0020954D400038B50546F6
:105000000C4BAA221A7012225A700222F0210A4C6A
:10501000A047012801D0002038BD064B0322BF2144
:105020002846064CA047012801D0002038BD014B7E
:10503000987838BD300F0020954D40004D4E40000F
:1050400010B50B462C227021014CA04710BD00BFAB
:10505000954D40002DE9F04182B000238DF80730D6
:10506000012906D002291ED1114D804601200024BD
:105070000BE0104DF9E70DF10703024640460E4ED6
:10508000B0473C44E4B20134E4B201280CD12346D9
:105090002F5D4FB1621CA95C012FECD902332B4468
:1050A000781EC0B2E9E7002002B0BDE8F08100BF81
:1050B0000C014100C4014100954D400010B51B4B4F
:1050C00000221A725A729A724FF4487199806421C0
:1050D000D9801A805A80164B98470121154B984762
:1050E000012802D0114B187A10BD01220F4B1A7201
:1050F0000F4B98470521104B9847034650B10B4A78
:105100005372002BEED00A4B98470C4B9847074B35
:105110005880E7E7064CA0470021064B9847A04778
:105120000321054B98470346E9E700BF700F0020B5
:1051300019C34000B9514000CD5340005D534000B9
:10514000014B187A704700BF700F002008B5114B53
:105150001B7A6BB90F4B9B7A8BB10E4A11889388DF
:10516000D2889B1A994214DC00220A4B9A7208BD1D
:10517000094B9847094B9847064B1880EAE7054AC0
:1051800011889388D2881344994202DB0122014B93
:105190009A7208BD700F002019C34000ED52400004
:1051A000014B987A704700BF700F0020014B1888A0
:1051B000704700BF700F002030B587B005460C4621
:1051C00000238DF8073072228DF808208DF80B30FF
:1051D00001228DF809208DF80C200DF107020492B0
:1051E00002228DF80A2005933C4B9847322202A9EF
:1051F00028463B4B9847002C3BD1012402238DF8D5
:105200000A3080238DF80B3001238DF807309C4243
:105210003CD08F238DF80B3003238DF80A30012CFE
:105220003BD09DF8073003F0F00343F002038DF804
:10523000073002238DF80A30012C35D007238DF872
:105240000730F9238DF80B30012C34D005238DF86D
:10525000073080238DF80B30012C33D02846214BAA
:105260009847012C35D000221F4B1A70204607B0FA
:1052700030BDA8238DF80B3001238DF80730322282
:1052800002A92846164B98470446B7E7322202A9DE
:105290002846134B98470446BBE7322202A928460A
:1052A0000F4B98470446BCE7322202A928460C4B14
:1052B00098470446C2E7322202A92846084B98477D
:1052C0000446C3E7322202A92846054B9847044604
:1052D000C4E70122044B1A70C8E700BF0168400010
:1052E0002D68400015684000E10B002030B587B004
:1052F00004460023059301AB049372238DF8083014
:1053000001238DF809309C238DF80B3002238DF892
:105310000C3003238DF80A300C4B9847322202A937
:1053200020460B4B9847054620460A4B9847012DCF
:1053300004D00020084B187007B030BD9DF8040061
:105340009DF8053000EB032080B2F5E701684000CE
:105350002D68400015684000E10B002030B587B093
:1053600004460023059301AB049372238DF80830A3
:1053700001238DF80930C0238DF80B3002238DF8FE
:105380000C3003238DF80A300C4B9847322202A9C7
:1053900020460B4B9847054620460A4B9847012D5F
:1053A00004D00020084B187007B030BD9DF80400F1
:1053B0009DF8053000EB032080B2F5E7016840005E
:1053C0002D68400015684000E10B0020F0B587B063
:1053D0000646002305930DF10703049372238DF80D
:1053E000083001248DF80940D9238DF80B308DF851
:1053F0000C4002238DF80A304901C9B241F0100176
:105400008DF80710204B9847322202A930461F4BD7
:1054100098470546D7238DF80B308DF80740A042FA
:105420000BD030461A4B9847DC238DF80B30032302
:105430008DF80A300024274608E0322202A93046BF
:10544000124B98470546ECE70134A4B2012D18D160
:10545000BFB9092C15D819200E4B984730460A4B76
:105460009847322202A93046084B984705463046F5
:10547000074B98479DF8073013F0010FE4D0012740
:10548000E2E7384607B0F0BD016840002D684000F3
:105490001568400015B74000F0B587B004460E46C9
:1054A000234B9847002304938A238DF8043001236B
:1054B0008DF805308DF808300DF11703039334276C
:1054C0008DF8077002238DF8063033788DF8173089
:1054D000322201A92046174DA8478DF8077033786E
:1054E0008DF81730322201A92046A8478DF80770A1
:1054F00033788DF81730322201A92046A84735238A
:105500008DF8073073788DF81730322201A92046C4
:10551000A84736238DF80730B3788DF8173032223C
:1055200001A92046A8472046034B984707B0F0BD85
:10553000016840002D68400015684000F0B587B054
:105540000446002505958A238DF8083001268DF83C
:1055500009608DF80C600DF1070304932B4B9847FD
:1055600055238DF807308DF80B5002238DF80A3043
:10557000322202A92046264DA84703238DF8073082
:105580008DF80B60322202A92046A8478DF80760EB
:1055900004238DF80B30322202A92046A8470723A6
:1055A0008DF8073030238DF80B30322202A92046C7
:1055B000A8470F278DF8077031238DF80B30322262
:1055C00002A92046A8478DF8077032268DF80B6097
:1055D000324602A92046A8478DF8077033238DF87C
:1055E0000B30324602A92046A8472046094B98476F
:1055F000094B1B68ADF804301B0C8DF8063001A96F
:105600002046064B984707B0F0BD00BF0168400038
:105610002D684000156840005C024100995440002C
:1056200030B587B0054610238DF808302022554B41
:105630001A630A20544B98472846544B9847002336
:105640000593E7238DF80B300DF107030493012335
:105650008DF80C308DF8093003238DF80A30322292
:1056600002A928464A4B984704469DF8073043F064
:1056700001038DF8073002238DF80A30012842D04B
:1056800006238DF80B3003238DF80A30012C41D00E
:105690009DF8073063F07F038DF8073002238DF803
:1056A0000A30012C3DD000238DF807300C238DF8F3
:1056B0000B30012C3CD00D238DF80B30012C3ED04B
:1056C0000E238DF80B30012C40D00F238DF80B30BA
:1056D000012C42D0E7238DF80B3003238DF80A30DC
:1056E000012C41D09DF8073023F001038DF80730DD
:1056F00002238DF80A30012C3DD02846254B9847CF
:10570000204607B030BD322202A92846204B9847D8
:105710000446B5E7322202A928461D4B98470446A5
:10572000B6E7322202A92846194B98470446BAE741
:10573000322202A92846164B98470446BBE732227C
:1057400002A92846124B98470446B9E7322202A91B
:1057500028460F4B98470446B7E7322202A928464D
:105760000B4B98470446B5E7322202A92846084B5E
:1057700098470446B6E7322202A92846044B9847C8
:105780000446BAE700100E4015B74000016840001B
:105790002D6840001568400030B587B004460D46BE
:1057A00000220592A8238DF8083001238DF80930D6
:1057B0008DF80B200DF1070204928DF80C300223B6
:1057C0008DF80A30124B9847012D0ED0022D15D0BE
:1057D00000238DF80730322202A920460D4B98474E
:1057E00020460D4B984707B030BD03238DF8073096
:1057F000322202A92046074B9847F1E702238DF891
:105800000730322202A92046024B9847E8E700BF42
:10581000016840002D6840001568400030B587B031
:1058200072238DF8003001238DF8013000238DF8AC
:1058300002308DF8033008228DF8042004AA029269
:1058400003938DF81000C0F307238DF81130C0F3D7
:1058500007438DF81230000E8DF813008DF81410E8
:10586000C1F307238DF81530C1F307438DF81630C7
:10587000090E8DF81710084CA047084B9847A04711
:1058800032226946064B98470546A047054B984784
:10589000284607B030BD00BF11C34000016840007A
:1058A0002D6840001568400030B587B00D46722362
:1058B0008DF8043001238DF8053000238DF8063073
:1058C0008DF8073004228DF8082005AA039204936E
:1058D0008DF81400C0F307238DF81530C0F307438B
:1058E0008DF81630000E8DF81700184CA047184B95
:1058F0009847A047322201A9164B98470446012831
:1059000008D0124B9847144B9847012C0DD02046D5
:1059100007B030BD01238DF806300C4B984732227A
:1059200001A90C4B98470446EBE79DF814309DF80D
:10593000152003EB02239DF8162003EB02439DF88C
:10594000172003EB02632B60E1E700BF11C34000A7
:10595000016840002D684000156840002DE9F043C3
:1059600083B080460F4691461BB11E46002501209C
:105970001CE0012001282BD0012833D0012836D08B
:10598000012839D04FF40003019308243FE0EA18BE
:10599000B25C4FEAC30E02FA0EF211440133DBB2DD
:1059A000A342F4D301280CD02544EDB2AC46BD424D
:1059B000E0D27C1B042C28BF0424E4B20023194647
:1059C000EEE70CF1201000F580701A4B9847EBE7DA
:1059D0004FEA084101F4FE0101F500011648154B9C
:1059E0009847C9E739461548124B9847C6E74946D4
:1059F0001348104B9847C3E7F22112480D4B9847C4
:105A0000C0E701A90C48104B9847013CE4B20128BB
:105A100004D11CB1019B13F4000FF2D118B9052079
:105A200003B0BDE8F0830CB90620F9E79DF8070044
:105A3000F6E700BF1D5840001001200018012000AB
:105A400014012000FC002000A958400010B582B0CD
:105A5000094B93E8030000908DF804106B46002278
:105A600005210120054CA047034610B90121044A35
:105A70001170184602B010BD600241005D5940002F
:105A8000E20B002038B50D460023024604213120E8
:105A9000064CA047044608B1204638BD29460448B4
:105AA000044B98470128F7D00524F5E75D594000DD
:105AB00020012000A958400010B582B08DF80410D4
:105AC0000B0A8DF805300B0C8DF80630090E8DF899
:105AD000071001AB024604212120024CA04702B06E
:105AE00010BD00BF5D59400008B5044B1B780BB1D9
:105AF000002008BD024B984708BD00BFE20B002004
:105B00004D5A40002DE9F04383B059B1012904D02A
:105B10000124204603B0BDE8F08340F65D0740F65F
:105B2000050503E040F2DD7740F2857580464FF0D1
:105B300000094C4601E0002CEBD1BD42E9D225F032
:105B40000306002CF7D101A93046164B98470446AE
:105B50000028F0D1019B8DF80030C3F307228DF8A7
:105B60000120C3F307428DF802201B0E8DF803308D
:105B7000E9B2F3B2C91AC9B2C1F10403BE1B9E4215
:105B800028BF1E46042E28BF0426F6B232466944BA
:105B900008EB0900044B984735444E445FFA86F9F8
:105BA000C9E700BF855A400091D7400028B10128BD
:105BB00001D000207047094800E0094800B583B0D3
:105BC00001A9084B984728B9019B13F4006F02D034
:105BD000012000E0002003B05DF804FB4000350028
:105BE00040003100855A400010B52DED028B82B087
:105BF000044601A93548364B98470346F8B14BB3E4
:105C0000002B32D0002B3BD0DFED328A002B49D065
:105C10009FED308A73B9DDED017AB8EE677AC8EE90
:105C2000077A9FED2D7A67EE877AFCEEE77A17EE1A
:105C3000902A6281184602B0BDEC028B10BD02A909
:105C400051F8043D23801B0C63802448204B984767
:105C50000346D4E702A951F8043DA3801B0CE3805E
:105C60001F481B4B98470346CAE702A951F8043D59
:105C700003F01F0323721B48154B98470346C1E7E7
:105C800002A951F8043DC3F3094308EE903AF8EE37
:105C9000688A9FED158A68EE888A14480C4B9847ED
:105CA0000346B3E702A951F8043DDBB208EE103A0F
:105CB000B8EE488A28EE888ADFED077A28EE278A30
:105CC0000B48034B98470346A4E700BF3008220067
:105CD000855A4000000000000000C8423808220039
:105CE000540822000800200000401C46040822003E
:105CF0001408220010B582B080230093054B1522B2
:105D000014210548054CA04710B1002002B010BD79
:105D10000120FBE77C0F0020000A0E40010000205C
:105D200008B5002213210348034B9847B0FA80F0CE
:105D3000400908BD000A0E40C5A1400010B5EFF3B0
:105D4000108404B972B6002308E09A0002F58002BC
:105D50000A4951F82310116001339BB27F2BF4D90B
:105D6000002212210648074B9847C0B204B962B618
:105D700008B1002010BD012010BD00BF7C0F002025
:105D8000000A0E40C5A1400010B400240EE04000FF
:105D900080F00700C0B20133DBB2072B05D810F04A
:105DA000800FF4D14000C0B2F5E70134944204D230
:105DB00011F8013B58400023EFE75DF8044B7047B2
:105DC00008B5094B1B781BB1022B01D0074808BD51
:105DD000074B9847012804D10122034B1A7003484E
:105DE00008BD002008BD00BFE30B00207C0F002091
:105DF000F55C400008B5094B1B781BB1022B01D0A4
:105E0000074808BD074B9847012804D10122034BDE
:105E10001A70034808BD002008BD00BFE30B002036
:105E20007C0F0020F55C4000A8B108B50346B1F531
:105E3000007F12D28818B0F5007F01D9002008BD7C
:105E400008461946064B1844064B98470222064B53
:105E50001A70012008BD00207047002008BD00BF57
:105E60007C0F002091D74000E30B002008B5064BC3
:105E70001B78022B01D0002008BD044B9847012855
:105E8000FAD1034B984708BDE30B0020215D400089
:105E90003D5D400090B110B504460268094B9A423E
:105EA00001D0002010BD9A220146FF20064B9847E2
:105EB00094F89A30984203D0002010BD002070471B
:105EC000012010BD5FE1AD5A895D40002DE9F84326
:105ED00005460E4617460A469C211E4B9847044627
:105EE000451B40B1731B052B05D94378552B07D0B3
:105EF00010237B7001E000237B702046BDE8F8830F
:105F000090F80280C37888EA0303FF2B02D01123A4
:105F10007B70F2E790F80490437909EB03291FFAAC
:105F200089F9B9F13A0F06D84D440635AE4205D28B
:105F300000237B70E1E712237B70DEE74A46811D78
:105F4000381D054B9847A7F8029087F80080012379
:105F50007B70D2E7F1D6400091D7400010B553884E
:105F60009C1D8C4219D83A2B01D9002010BD114636
:105F70009C23037055234370137883701378DB439D
:105F8000C3709378037153881B0A4371528804319C
:105F90000630034B9847012010BD002010BD00BF04
:105FA00091D7400070B582B0044603784C3B0C2B6F
:105FB00000F2A780DFE803F007A5A5A5A5A5A5A584
:105FC000A52476518E004388032B05D0504B002228
:105FD0005A8082221A7099E003798DF8043043794F
:105FE0008DF8053083798DF806304A4B984701A922
:105FF000494B9847464B00225A8081221A7085E00F
:106000004388012B05D0424B00225A8082221A700D
:106010007CE003790F2B05D93D4B00225A80822268
:106020001A7073E03D4B9847394A5523137020236B
:106030005380237900EB4310066845688468C16883
:1060400056609560D4601161066945698469C169CB
:1060500056619561D461116258E04388212B05D0C7
:106060002B4B00225A8082221A704FE001790F29AF
:1060700005D9274B00225A8082221A7046E020223E
:1060800049010530264B9847012805D0204B0022B6
:106090005A8082221A7039E01D4B00225A808122D8
:1060A0001A7033E043882BB1194B00225A808222A8
:1060B0001A702BE01B4B9847012805D0144B002287
:1060C0005A8082221A7021E0114B00225A808122CC
:1060D0001A701BE043882BB10D4B00225A8082229C
:1060E0001A7013E0104B984728B9094B00225A80C8
:1060F00081221A700AE0064B00225A8082221A700E
:1061000004E0034B00225A8082221A7002B070BD54
:106110007C11002019C3400099544000F55D4000F7
:10612000295E40006D5E4000E95A4000004870471B
:106130007C110020F0B583B0EFF31083B3FA83F342
:106140005B09019372B6BFF35F8F0022364B1A7062
:10615000019E364B1B68364A15682B447F2B2AD884
:10616000324B1C682246334933482844334B984706
:106170002C442F4B1C6000222C4B1A602EB10122A4
:10618000294B1A70BFF35F8F62B62D4A284B1968EE
:1061900029482C4B98470146D0B1274BC31A2848B1
:1061A00042881A44951D4478012C15D044BB802B9D
:1061B0001CD900242AE01D4A136814682C441B1BB8
:1061C00003F18004204A137843F001031370C9E7F8
:1061D0000024174B1C6019E01748154F3E68761BCA
:1061E00032464119194B98473E600FE0104D2C681C
:1061F000E41A22461048154B98472C60002405E00D
:106200000633802B05D90024094B1C60204603B0BF
:10621000F0BD0948064D2C68E41A2246C1180B4B04
:1062200098472C600024F1E7FA010020C4140020F4
:10623000D41400201C150020C413002091D7400066
:10624000D8140020CD5E4000D0140020C5D84000F6
:1062500010B5184B9847184B18600DE0174B195D97
:106260001748184B98470134E4B2174B1B689C42FF
:10627000F4D30022144B1A604FF0FF310120134B6E
:106280009847134B98470128F6D11248124B98476C
:10629000124B9847024680210848114B9847012825
:1062A000EAD10E4B984743880633074A136000240F
:1062B000DBE700BFADB94000C81400204414002043
:1062C000008201404FA64000CC140020C5BB400016
:1062D00035614000D8140020A55F40002D614000CA
:1062E0005D5F400030B583B08024224600211B480A
:1062F0001B4DA847224600211A48A84700231A4AE6
:1063000013601A4A13601A4A13701A4A1021516610
:10631000C2F8901051655162C2F88010116F21F0DF
:1063200010011167516F21F010015167124A4FF4AB
:1063300000211160202182F8131301210F4A91607E
:106340000193009322460E490E480F4CA0470128A6
:1063500002D00E480E4B984703B030BD1C150020EC
:106360008DD9400044140020C4140020CC14002017
:10637000D0140020000E0E4000E100E00082014039
:1063800068024100516240005DB44000700241006B
:106390003DD14000194B1B6913F0010F2DD0174B55
:1063A0005B6913F0010F28D000B583B0144B1B6854
:1063B0007F2B1CD8124A1368591C11600F4A91692F
:1063C000104AD15402A9002341F8043D0E4B18682D
:1063D0000E4B9847019B3BB14FF080520C4B1A601B
:1063E000BFF34F8FBFF36F8F03B05DF804FB094A13
:1063F000137843F001031370E4E770470082014013
:10640000C41400201C150020C814002031BD400019
:1064100004ED00E0D0140020154B98421BD003F58A
:10642000A033984219D003F58043984217D0A3F5C2
:106430004043984215D003F58043984213D0A3F50A
:10644000A033984211D003F56033984201D0322036
:1064500070471620704708207047092070470E20AB
:10646000704713207047142070471520704700BFF5
:1064700000C000404900B0FBF1F00338002302E007
:1064800040080133DBB2FF28FAD8020202F47F424F
:1064900052FA80F01B0403F4E02318447047000014
:1064A0002DE9F843D0F80090037ADBB2012B00F01D
:1064B0009E80044609F5C065087908B9BDE8F883EF
:1064C00017460E46012323720023E371E1604C4B13
:1064D00098478046B378022B08D07378012B18D0E8
:1064E00033781B0403F4FE036B603DE07378012BEB
:1064F00009D033781B0403F4FE0303F580736B604B
:10650000F378EB6030E033785B081B0403F58073AD
:10651000F5E733785B081B04E6E70323A371002348
:106520002372237A002B65D02B6A13F4807F3BD132
:1065300013F0040F3CD1324B984708EB0703984205
:10654000F2D90523A371002323722E4BC9F800361C
:106550002EE00423A37100232372E2E7284B98471F
:1065600008EB0703984217D83379E2799B1A002B7E
:10657000D7DD2B6A13F4807FCFD113F4007FE8D1ED
:1065800013F0040FEAD0B168E379DBB25A1CD2B23F
:10659000E271CB5C6B63E1E70523A37100232372F7
:1065A000184BC9F80036BCE70323A37100232372FC
:1065B000237A13B30223C9F800362B6A13F0010FB4
:1065C0000ED10F4B984708EB07039842F5D90523E6
:1065D000A371002020720B4BC9F80036BDE8F88388
:1065E000002323720223A3710120BDE8F883002059
:1065F000BDE8F8830020BDE8F88300205EE700BF17
:10660000F16A4000028000052DE9F84FD0F800A0A3
:10661000037ADBB2012B00F09E800AF5C0660B798D
:1066200013B91846BDE8F88F17460D4604460123F6
:1066300003720023C371E160494B98478046AB78F1
:10664000032B14D06B78012B24D02B781B0403F47C
:10665000FE0303F58053736095F80490B9F1010FC0
:106660001ED00123CAF800364FF000094DE06B78C8
:10667000012B09D02B781B0403F4FE0303F5885388
:106680007360EB78F360E7E72B785B081B0403F596
:106690008853F5E72B785B081B0403F58053DAE792
:1066A0000323CAF8003630E00323A37100232372CA
:1066B000237A002B51D0336A13F0010F45D1284BB8
:1066C000984708EB07039842F5D90523A3710023E7
:1066D0002372244ACAF80026A3E70423A3710023E7
:1066E0002372E5E70523A371002323721D4BCAF82B
:1066F0000036DDE71BF0020F07D0A968E379DBB2B3
:106700005A1CD2B2E271326BCA54E379DBB22A79F5
:106710009342CDD2D6F820B01BF4807FC4D11BF4B5
:10672000007FDAD10E4B984708EB07039842D9D87F
:10673000B9F1000FDED12B79E2799B1A012BD9D167
:10674000022333604FF00109D4E7002323720223B0
:10675000A371012365E7002363E7002361E700BF1E
:10676000F16A4000028000052DE9F04106468846A6
:10677000046820461B4B9847312801D9BDE8F081B9
:106780000546194B9847032323602423C4F8003699
:1067900041461648164B9847C4F81006002333723A
:1067A0000123B3716BB2002B07DB5A0905F01F0000
:1067B000012181400F4840F82210002B0BDB03F130
:1067C000604303F56143202283F8002301200A4B34
:1067D00098473061D2E705F00F05084B20225A5543
:1067E000F4E700BF1964400065A440000000DC0528
:1067F0007564400000E100E0E5AF400014ED00E00A
:1068000008B54FF0FF310069014B9847C0B208BD91
:1068100005B0400010B500231A4619460069024C25
:10682000A047C0B210BD00BFADAE400008B583792F
:1068300063B18B78032B0BD8DFE803F00205020568
:10684000044B984708BD044B984708BD002008BD7D
:10685000002008BDA164400009664000F8B5064666
:10686000036803F5C064256AC76815F0040F0BD0F0
:10687000E26A12F0040F07D0BA78002A4DD0022A3B
:106880004BD0BA78032A5ED015F0020F08D0E26A26
:1068900012F0020F04D0BA78012A73D0032A71D003
:1068A00015F4807F0DD0E36A13F4807F09D040F2A5
:1068B0000733A362002333720323B371FB6803B170
:1068C000984715F4007F0DD0E36A13F4007F09D0D8
:1068D00040F20733A362002333720423B371FB68D1
:1068E00003B1984715F0010F16D0E36A13F0010FBA
:1068F00012D0BB780BB1022B09D140F20533A36251
:10690000002333720223B371FB6803B19847BB784D
:10691000012B54D0032B52D0F8BDF279D2B2397981
:106920008A4208D2B868F279D2B2511CC9B2F17168
:10693000825C6263A5E70222C3F80026012262623C
:106940000422A2629DE77A78012A11D03A781204D3
:1069500002F4FE0202F5805262603A79012A0DD0FB
:106960000122C3F800260422A262022262628BE79F
:106970003A785208120402F58052EDE70322C3F878
:106980000026F0E7B868F279D2B2511CC9B2F171B1
:10699000216B8154F179C9B23A79013A91420AD016
:1069A000F379DBB23A7993427FF47AAF01236362E1
:1069B0000223A36274E70222C3F80026F0E740F244
:1069C0000333A362002333720223B371FB68002BED
:1069D000A2D09847A0E7000070B4056805F5C0662E
:1069E0000379202B0BD9A3F12001CBB21A4C012142
:1069F00099402160216521612163002211E0174C3B
:106A0000F5E701339BB2B3F52F7FFAD3616300231F
:106A100001E001339BB2B3F52F7FFAD3216301323A
:106A2000D2B2092A01D80023EDE7616161603269C1
:106A30008023C5F80036002301E001339BB2B3F593
:106A40002F7FFAD332612423C5F800360023037266
:106A50000123837170BC704700100E40000E0E4081
:106A6000F8B5084C4FF4804666630A20064DA847E7
:106A7000402767630A20A84727630A20A8472663A0
:106A8000F8BD00BF000E0E4015B74000F8B578B94C
:106A9000114D4FF480736B630220104CA0474FF0F0
:106AA00080736B630420A04701220D4B5A63F8BD2D
:106AB000094E4FF480737363094F02253D632846E6
:106AC000064CA04701233B630420A0474FF080738E
:106AD00033632846A047F8BD000E0E4015B74000AE
:106AE00000100E400322014B1A60704730140E4014
:106AF000044B986801E0034B9868024B9B689842EE
:106B0000F9D1704730140E40014B1880704700BF18
:106B10009C15002008B5154B1B8807EE903AF8EE3F
:106B2000677A9FED137A67EE876AB7EE007A37EEE1
:106B3000667A9FED106AC6EE276A66EE877A17EED0
:106B4000900A0D4B9847DFED0D7A07EE100A27EEFD
:106B5000277ADFED0B7A77EEC77ADFED0A6A86EEE9
:106B6000A77A094B83ED007A08BD00BF9C15002071
:106B700001088039FFEF7F457DC340003313954303
:106B800000F05745C47D7B49A0150020BFF35F8FFF
:106B9000024B1868BFF35F8F704700BFA01500203D
:106BA0008388B3F59F5F04D0B3F5706F0ED00020DB
:106BB0007047C288B2F51F6FF6D14289A2F5E7523D
:106BC000093A92B2C62AEFD801207047C388B3F5BC
:106BD000F06F01D0002070474389A3F50B53053BAC
:106BE0009BB2C62B01D802207047002070470000DE
:106BF00008B5044B98476420034B9847034B9847CC
:106C0000F7E700BFF944400015B74000156B40009E
:106C10002DE9F041944B9847944B1860944B98475A
:106C2000944B98470222944B1A63944B984705461D
:106C3000002407E00520924B9847904B9847054663
:106C40000134E4B20DB9132CF4D98E4B9847294680
:106C50008D4B98478D4B984740F21310884B9847BF
:106C60008B4B9847002416E0A2008A4911F8243083
:106C7000501C085C03EB0023901C085C03EB0043F2
:106C80000332895C04F5406003EB01618000824BB4
:106C900098470134A4B23F2CE6D901207F4B984796
:106CA0001920774B98474FF48072734B1A637C4BD3
:106CB00098476F4B98477B4B98477B4B98470546C7
:106CC0007A4B9847044678B901246B4BDB6B13F47D
:106CD000004F16D0764B98470F20764B98470146C9
:106CE0006548754B984726E105F19406604B984737
:106CF0003146724B984795F89830002BE5D0002428
:106D0000E3E76F4B9847E7E700206E4DA8476E4BCF
:106D100018700120A8476D4B187016E16C4B98470E
:106D200020B16C4B9847002840F0148100226A4B38
:106D30001A70514D4FF480766E631920504B98476E
:106D40002E6307E1634B9847002800F00881624BEF
:106D50001B78002B40F006810020604EB047604D4C
:106D600028700120B0475F4B18702B78002B00F083
:106D7000F980002800F0F6800127574B1F705A4D0C
:106D800028465A4B98472846594B984780464FF417
:106D9000FA703B4B98470020B047514D2870384659
:106DA000B047504B18702B7803B118B900224A4BEA
:106DB0001A70D7E0414600204E4DA847414638465C
:106DC000A8474D4D002128464C4B98472B78112B56
:106DD00015D0002108464A4DA84700210120A847A8
:106DE0003CB3484B984720B3474B1B78CBB10121AC
:106DF0000020464DA84701210846A847B2E06B781D
:106E0000002BE6D1AB78002BE3D1EB78892BE0D1D6
:106E10002E46294600203E4DA84731463846A84711
:106E2000D7E700210846394DA84700210120A8478F
:106E300098E001210020354DA84701210846A847C8
:106E400090E00021334B19702B482C4B98478EE073
:106E50000020314B1870214DA847214B187001209C
:106E6000A847204B187087E0ADB94000F40B002014
:106E700019C3400021564000000E0E405945400005
:106E800015B7400011C3400099574000616A4000A7
:106E90004D5A400090024100B95A40008D6A4000AE
:106EA000BD5040003D554000C15D4000955E400032
:106EB000714D400043A040001FA040009954400085
:106EC0004D4D4000FD4F4000B1000020B2000020B9
:106ED00065C3400071C34000E80B0020AD5B40007B
:106EE000E60B0020E70B00207C160020E95B400049
:106EF000A16B40005550400024160020055B400067
:106F0000954F400041514000B3000020B94F400070
:106F100041504000E40B0020E50B00202C4B98472B
:106F200030B101222B4B1A702B4B1B78002B41D117
:106F30000A202A4B9847284B1B78002B7FF4E4AE9D
:106F40004723274A1370274A1370234B1B78002BC3
:106F50007FF4E4AE244B984700287FF4F3AE002280
:106F60001D4B1A70214B1B78002B7FF46AAF204B0E
:106F70001B78002B7FF46CAF1E4B984710B31E4B51
:106F80009847002CD4D0134B1B78002BC6D0104B45
:106F900098470028CCD100220E4B1A700E4B1B785C
:106FA000002BC5D011461046144DA84700210120E2
:106FB000A847BDE711460020104DA847012108460B
:106FC000A847B5E70E4B98476420044B9847B2E7B3
:106FD000A1514000B3000020E80B002015B740008D
:106FE000B1000020B200002065C34000E40B002087
:106FF000E50B0020415140004D514000B94F400089
:10700000BD50400008B5284B9847284B186006E053
:1070100000210846264CA04700210120A0474FF040
:10702000FF310120234B9847234B1B78013B062B54
:10703000F5D801A252F823F05570400011704000BD
:107040007770400087704000657040009770400086
:10705000A370400001210020154CA04701210846E3
:10706000A047DCE7154D29880020154CA04729884A
:107070000120A047D3E700210846124CA047002179
:107080000120A047CBE7012100200E4CA0470121A1
:107090000846A047C3E70C4B98470C490C4B984750
:1070A000BDE70C4B9847BAE7ADB94000EC0B0020A8
:1070B000DD4F4000C5BB4000A7150020881600200A
:1070C000454F4000B94F400019C34000A4150020AF
:1070D000995440006D5E4000F8B5524B9847524BB2
:1070E00018604FF47A72514B1A80402200215048A8
:1070F000504B984734E0504B98474D4A55231370F6
:10710000202353704D4B1B7800EB431007684668F3
:107110008568C168C2F80270C2F80660C2F80A50F9
:10712000C2F80E10076946698569C169C2F8127014
:10713000C2F81660C2F81A50C2F81E101AE03C4895
:107140004D2303703E4B1A7842701A783D49023045
:107150003D4B984710E0402200213548354B984779
:10716000324B198889B20120384B9847044658B1F0
:107170005528C0D04D2CE2D0354B98470028EAD096
:107180002B48344B9847E6E7294C232323701423DC
:107190006370314B9847C0F30F23A370E0702F4BFF
:1071A0009847C0F30F23237160712D4B9847C0F3AC
:1071B0000F23A371E0712B4B9847C0F30F23237269
:1071C0006072294B9847C4F80A00284B1B7807EED9
:1071D000103AB8EE477A9FED266A27EE067ADFED81
:1071E000256A37EE667A17EE103AC4F80E30224B55
:1071F0001B7807EE903AF8EE677A67EE867A77EEBC
:10720000E67A17EE903AC4F81230114B984728B935
:10721000402200210648074B9847A1E720460D4B26
:107220009847F5E7ADB94000F00B0020221600208A
:10723000CC1500208DD94000F55D400020160020BF
:10724000211600208C16002091D74000C5BB4000BD
:1072500039C3400045764000E14C4000AD5140004C
:10726000414540004D4540008D6B4000B10000207D
:10727000B4C8363F6FDB4A42B200002010B582B07E
:1072800000230193012200928022194919481A4CC7
:10729000A047012802D01948194B984700230193B1
:1072A00003220092802217491748134CA047012857
:1072B00002D01648124B9847002301930093802276
:1072C000134914480C4CA047012802D012480C4B1B
:1072D0009847002301930093802210491048064CE0
:1072E000A047012802D00F48054B984702B010BDB7
:1072F00090034100D97040005DB440009803410004
:107300003DD14000BC03410005704000C003410076
:10731000DC034100116C4000E8034100100441000F
:10732000F16B40001404410030B585B00446037889
:10733000532B25D02378472B2CD02378672B37D09D
:107340002378462B3CD02378522B3DD02378502BEA
:1073500044D02378492B64D02378422B7ED0552B00
:1073600000F08E802378572B00F0A8802378562BCE
:1073700000F0AE8023784C2B00F0C28005B030BD09
:1073800043781BB901206E4B9847D3E700206C4B24
:107390009847CFE76378A07800EB032080B210F421
:1073A000004F02D1674B9847C7E747F6FF70F9E7F0
:1073B0006378A07800EB032000B2634B9847BFE7E7
:1073C0006078624B9847BEE76278A37803EB0223AC
:1073D0009BB2092BBAD95E4A1380B7E76378B3B979
:1073E00002225C4B1A7004A9002341F8043D5A4B59
:1073F00018685A4B9847039B002BAAD04FF0805235
:10740000574B1A60BFF34F8FBFF36F8FA1E7012B6C
:1074100003D000224F4B1A70E5E701224D4B1A7042
:10742000E1E76278A37803EB02234E4A138005223A
:10743000484B1A7004A9002341F8043D464B1868D4
:10744000464B9847039B002B86D04FF08052444B0D
:107450001A60BFF34F8FBFF36F8F7DE7424BBB22A4
:107460001A601A225A60BFF34F8F4049CA6802F46B
:10747000E0623F4B1343CB60BFF34F8F00BFFDE78C
:1074800063780F2B3FF66EAF3A4A1370002304AABD
:1074900042F8043D38490868009203225521374DCF
:1074A000A847039B002B3FF45DAF4FF080522C4B5D
:1074B0001A60BFF34F8FBFF36F8F53E761780F29C7
:1074C0003FF654AF20224901A01C2D4B98474DE7B1
:1074D0000722204B1A7004A9002341F8043D1E4BDB
:1074E00018681E4B9847039B002B3FF443AF4FF0A7
:1074F00080521B4B1A60BFF34F8FBFF36F8F39E77A
:10750000204B62781A70A2785A70E2789A7006223C
:10751000104B1A7004A9002341F8043D0E4B186863
:107520000E4B9847039B002B3FF428AF4FF080523F
:107530000B4B1A60BFF34F8FBFF36F8F1EE700BF77
:10754000457940000D79400039794000954C400064
:1075500022160020A7150020EC0B002031BD4000B2
:1075600004ED00E08816002090140E4000ED00E0CD
:107570000400FA0520160020F00B002049BC400052
:10758000295E4000A41500200023044A1370044A19
:1075900013700120034B1870704700BF000C0020CF
:1075A000FC0B0020F80B0020704700207047000003
:1075B0000D4B5B881A0A032A01D00020704713F094
:1075C000FF0F0ED1084BDB88402B01D00020704705
:1075D000054B064A9A60064A1A6140229A810120A8
:1075E00070470020704700BF381B0020040C0020AB
:1075F000257640000122014B1A707047F80B0020DD
:1076000010B5034B034A04490448054CA04710BD7C
:10761000B175400084010020FC0B0020000C00200C
:107620004577400008B5044B9B89402B00D008BD2E
:107630000248034B9847FAE7381B0020040C00204F
:1076400029734000224B1B780BB9184670472DE96F
:10765000F04184B00746EFF31083B3FA83F35B097C
:10766000039372B6BFF35F8F00211A4B1970DDF8D8
:107670000C80194D40222846184B98473C4640370D
:107680002E4620686168A268E3680FC6103435464C
:10769000BC42F5D1124B009340230F4A00218120B8
:1076A000104CA04780F00100094B1870B8F1000F92
:1076B00005D00122074B1A70BFF35F8F62B6044BEF
:1076C0001B7883F00103184604B0BDE8F08100BFC9
:1076D000F80B0020FA010020440C00208DD9400056
:1076E000F5754000359B400010B50446134B984794
:1076F000837A212B01D0002010BD00F10902104B2C
:107700005B881B0A212B04D0C27B93420BD0002044
:1077100010BD0B4B9A60427AD9888A4228BF0A462C
:107720009A81012010BD064B9C60028AD9888A424A
:1077300028BF0A469A81012010BD00BFE17F4000AA
:10774000381B0020F8B5264C247865B2002D07DBE5
:10775000002D40DB04F06004202C22D00020F8BD76
:1077600014F0600603D11E4F7F78062F0BD0202E19
:10777000EED11B4A5278022A09D0032A0CD0012AE2
:10778000E6D19847F8BD1046164B9847F8BD144B04
:10779000986001209881F8BD114B99600120988173
:1077A000F8BD0F4A52780A2A07D00B2A0BD0092AB3
:1077B00001D00020F8BD9847F8BD094B5B881B0A33
:1077C00003700120F8BD064BDB8833B9044B5B889E
:1077D0000B700120F8BD0020F8BD0020F8BD00BFEF
:1077E000381B0020E976400070B590B000248DF879
:1077F00035408DF836408DF837408DF839408DF89A
:107800003A40ADF83E400F238DF834300A23ADF8EE
:107810003C3001258DF838500DAA0B4907A80B4EB6
:10782000B0470DAA0A4901A8B0471023079A136070
:10783000019A1360074B1D70074B1C7047F6FF72CF
:10784000064B1A8010B070BD00C002404D9F400032
:1078500000000340840C00208C18002056190020E2
:1078600042B110B420B119B1034B586099605A80ED
:107870005DF8044B704700BF840C0020154B1B784B
:107880003BB3144B5B8823B3124A52680AB31149C5
:107890008968F1B1F0B583B0009201930E4D6A464C
:1078A000694628460D4FB8474FF480362E62094B83
:1078B0009B6800930A4C6A4669462046B847266290
:1078C00001212846074DA84701212046A84703B0BB
:1078D000F0BD7047840C002000C10240899E40002A
:1078E00000010340A19E4000064B1B783BB1054BB5
:1078F0005888054BD3F80431C01A80B27047002075
:10790000704700BF840C002000C00240094AD36DBC
:1079100023F4FF4323F07F03C0F30E000343D3653A
:1079200002F58042D36D23F4FF4323F07F03184315
:10793000D065704700C00240014B1880704700BFFF
:1079400056190020014B1870704700BF8C1800209A
:10795000004870475819002000487047AC160020B6
:10796000704770472DE9F8434C4B984705464C4B00
:107970009847044678E0A0EB070E1FFA8EFE0EF142
:10798000F00E1FFA8EFE7EE03121002308E02F2149
:10799000FBE744480078C0B2012831D001339BB2E4
:1079A000994252D9DA1992B2EF2A01D9F03A92B239
:1079B0003C4800780028ECD13B48B0F9000035F98C
:1079C000126006FB00F6F6134FEA8308DFF8E0C00A
:1079D0000CF8236008F10109C6F307260CF80960CA
:1079E00034F9122000FB02F2D21308F102000CF865
:1079F000002008F10308C2F307220CF80820CDE7A5
:107A000035F9120034F91220024402EBD2725210FE
:107A100012F5004F05DBB2F5004F03DB47F6FF72AE
:107A200000E0224A98005FFA82FC214E06F823C04B
:107A300000F10108C2F3072206F8082000F102084D
:107A400006F808C003303254A8E71A4BA3F800E048
:107A50007744BFB2184B1F80EF2F01D9F03F1F8032
:107A600089001348154B98474FF0FF310120144B04
:107A70009847144B9847104B1F88B842FFF47BAFD0
:107A8000C01B1FFA80FEBEF1300F3FF67DAFBEF186
:107A90002F0F7FF67CAF302177E700BF5179400090
:107AA000597940008C180020561900200080FFFFF3
:107AB0009018002054190020900C002055464000DA
:107AC000C5BB4000E9784000024B1B681B68588822
:107AD00018447047A00C002038B504460D46094BE9
:107AE0009847024620782044904207D24378042BDE
:107AF00006D0AB4205D003781844F5E7002038BD26
:107B0000002038BDC97A400038B5144B1B780BB340
:107B1000134B1B681B681A7982421DD90D46044617
:107B2000104A1360104B984703E01A7813440D4A2B
:107B300013600C4B1B6898420AD95A78042AF4D176
:107B40009A789442F1D1DA78AA42EED1012038BD78
:107B5000002038BD002038BD002038BD9C0C00201E
:107B6000A00C0020A40C0020C97A4000084BDB8840
:107B700063B9074B5B88012B01D000207047054A91
:107B8000138823F002031380012070470020704700
:107B9000381B0020920C002000207047044BDB882B
:107BA00023B9044A024B1A61012070470020704734
:107BB000381B0020D17E400038B5134B1B7803B32F
:107BC000124B1C79124B1B681B681B799C4201D31A
:107BD000002317E0002120460E4B9847034688B14A
:107BE0000B4B1B685B6853F82450EB6898470146C1
:107BF0002046084B9847034620B1AB689847034698
:107C000000E00023184638BD9C0C0020381B0020E3
:107C1000A00C0020097B400038B5104B1B78D3B175
:107C200000240F4B1B681A681279944211D25B68CA
:107C300053F82450EB68984701462046094B984773
:107C4000034648B1AB689847034628B90134E4B20B
:107C5000E7E7002300E00023184638BD9C0C002015
:107C6000A00C0020097B400070B504460021114B98
:107C70009847054608B9284670BD0F4B1B685B68DE
:107C800053F82460F368984701462046094B98470B
:107C900005460028EFD0094B1C6805212046084BFB
:107CA0009847044618B18078064B9847F5E7736803
:107CB0009847E0E7097B4000A00C0020A40C0020BE
:107CC000D97A4000B598400008B5064BDB88022BF6
:107CD00001D0002008BD02210348044B9847012031
:107CE00008BD00BF381B0020920C0020999740006F
:107CF00010B5154B9B78012B04D043B1022B0CD04F
:107D0000002010BD0720114C50B1002311E00421C8
:107D10000F48104B98470020F6E715200E4CF3E76C
:107D2000012010BDE15C0D4A02EB4302518001339A
:107D3000DBB28342F6D3411C4900C9B20748017047
:107D4000044B9847012010BD381B0020DC010020A7
:107D5000D801002099974000E4010020AC010020E8
:107D600008B5234B5B88DAB21B0A013B0E2B38D8CF
:107D7000DFE803F00817313737373737373737370A
:107D800037372A001B4B186801781B4B9847184B54
:107D9000DA889B899A4228D2154B9A81012318468A
:107DA00008BD144B1B685B7C9A4201D30023F6E7A5
:107DB000104B5B6853F8320041880F4B98470C4BCF
:107DC0009B6802225A70E2E70A4B986858B14188D2
:107DD000094B9847DBE7094B984703460028D6D163
:107DE000DDE70023DBE70023D9E70123D7E700BF66
:107DF000381B0020B400002099974000F17C40001F
:107E000008B5064BDB88012B01D0002008BD0121FD
:107E10000348044B9847012008BD00BF381B0020D1
:107E20009C0C00209997400038B5154BDB88012B3E
:107E300002D00024204638BD124B1B78F3B1104B02
:107E40001D79114B1B681B681B799D4201D30024CF
:107E5000F0E7002128460D4B984704460028E9D05A
:107E6000094B1B685B6853F82530DB689847084B63
:107E7000187001211846074B9847DBE70024D9E723
:107E8000381B00209C0C0020A00C0020097B400027
:107E9000980C00209997400008B5094BDB88022B0D
:107EA00001D0002008BD064B1879064B9847064BB9
:107EB000188002211846054B9847012008BD00BFD5
:107EC000381B002005994000940C00209997400031
:107ED00008B5034B588800F07F00024B984708BD57
:107EE000381B00204197400038B505460F4B984796
:107EF0000346C0B10E4B1C68052120460D4B984728
:107F0000044640B18288C17880780B4B984703467D
:107F10000028F1D107E0094B1B685B6853F8253056
:107F20001B6898470346184638BD00BF097B4000D0
:107F3000A40C0020D97A4000A5974000A00C002096
:107F400038B50C4BDB8893B90B4B1B780BB900236E
:107F50000EE0084B1C799D782046084B9847034655
:107F600030B129462046064B9847034600E00023DF
:107F7000184638BD381B00209C0C0020697C40004E
:107F8000E97E400008B5074BDB884BB9054B5B88A1
:107F90000BB1002008BD034B1879034B984708BD6F
:107FA000002008BD381B0020419A4000094BDB88A7
:107FB0006BB9084B5B880BB10020704710B5054CBE
:107FC0002079054B98472079044B984710BD002035
:107FD000704700BF381B0020B19C40004999400009
:107FE000014B1868704700BFA40C002008B5014B76
:107FF000984708BD7D96400010B50B4B1B7863B1C8
:10800000002404E02046094B98470134E4B2084BB1
:108010001B681B681B799C42F4D30022024B1A7028
:108020000122044B1A8010BD9C0C0020697C40008A
:10803000A00C0020920C00201C4BDB8813B1002305
:108040001846704710B51A4B984750B3174B9A789B
:10805000184B1B685B7C9A4201DD002322E0164B23
:108060009847124B9B78154A1370EBB1114A52682E
:1080700003F10053013B02EBC303114A13600024D8
:108080000F4B1B681B681B799C4208D200212046BD
:108090000C4B9847034628B10134E4B2F0E70123C2
:1080A00000E00023184610BD0123FBE7381B002029
:1080B0007D974000B4000020F97F40009C0C002018
:1080C000A00C0020E97E400008B5344B1B7813F06B
:1080D000800F0ED113F01F0343D1304A5278013A7A
:1080E000082A3ED8DFE802F0343D373D313D3D3DC2
:1080F0003A002A4AD288002A4ED013F01F0306D134
:10810000264A5278062A0BD0082A0CD02AB1012B15
:108110000CD0022B11D0002008BD214B984708BD80
:10812000204B984708BD204B984708BD1B4A527802
:108130000A2AEED11D4B984708BD184B5B780BB14E
:10814000002008BD1A4B984708BD1A4B984708BD38
:10815000194B984708BD194B984708BD184B9847CD
:1081600008BD012B03D0022B08D0002008BD0B4A0C
:1081700052780B2AF7D1134B984708BD074B5B7811
:10818000012B03D0032B04D0002008BD0E4B9847D1
:1081900008BD0E4B984708BD002008BD381B0020C5
:1081A000C97C4000617D4000017E4000297E400086
:1081B000997E40009D7B40006D7B4000997B400094
:1081C00039804000417F4000857F4000AD7F400006
:1081D0000B4B1B7813B110B5002402E0704701343B
:1081E000E4B2084B1B681A681279944207D25B68A4
:1081F00053F824301B69002BF1D09847EFE710BDEE
:108200009C0C0020A00C002008B5184B00229A817D
:108210001A615A611B7813F0800F11D113F0600FAF
:1082200014D0124B1B7803F01F03012B14D00F4BFB
:108230001B7803F01F03022B14D00023184608BD3F
:108240000A4AD288002AE9D10023F7E7084B984769
:1082500003460028E5D0F1E7064B9847034600287F
:10826000E5D0EBE7044B98470346E7E7381B0020CF
:10827000C9804000B97B4000197C4000F8B5044635
:108280000E46114B984705462046104B984705402F
:1082900001D0002403E0F8BD0134062C11D88DB1C3
:1082A00023010B4AD058B042F6D102EB04135968AF
:1082B0000D42F1D01F46DB6898477B6825EA03052D
:1082C000EAE7F8BDF8BD00BF27A040002BA04000A2
:1082D000A80C0020F8B5164C2768062F26D80024D5
:1082E00001E00134E4B2A446A7420AD3114E2501AD
:1082F00006EB050E75598D42F3D1DEF80450954218
:10830000EFD1CEF80010CEF80420CEF80830069950
:10831000CEF80C100137BC4505D011461A46064B65
:1083200098470020F8BD02490F60F6E70120F8BD2C
:10833000180D0020A80C0020ED9F40002DE9F04111
:1083400082B004460F4690460A4B984705462046A1
:10835000094B984706462046084B9847CDF80080C1
:108360003B46024631462846054CA04702B0BDE8D0
:10837000F08100BF2FA040003DA0400043A040007E
:10838000D582400008B50B210148024B984708BD33
:10839000000E0E407D82400008B50C210148024BC2
:1083A000984708BD00100E407D824000F8B5064693
:1083B0000C461546224B984707464FF0FF31304692
:1083C000204B98473046204B9847002C0CDB630924
:1083D00004F01F0101228A4020331C4941F8232068
:1083E000BFF34F8FBFF36F8F002C08DB630904F0DE
:1083F0001F0101228A406033144941F82320002CD8
:1084000017DB2D01EDB204F1604303F5614383F8FE
:108410000053002C08DB620904F01F04012303FA57
:1084200004F40A4B43F8224039463046084B98473B
:10843000F8BD04F00F022D01EDB2064B9D54E8E7A4
:108440002BA0400023A0400027A0400000E100E056
:108450001FA0400014ED00E082B0024610B9244B8A
:108460001B783BB912B1224B1B780BB3204B1A700F
:1084700002B070471F4B1B7803B9FEE7EFF3108380
:10848000B3FA83F35B09009372B6BFF35F8F0021E9
:10849000194B1970009817490B78013B0B70002895
:1084A000E0D00121144B1970BFF35F8F62B6D9E79A
:1084B000104B1B78FF2B19D0EFF31083B3FA83F323
:1084C0005B09019372B6BFF35F8F00210A4B1970ED
:1084D000019808490B7801330B700028C6D00121A0
:1084E000054B1970BFF35F8F62B6BFE7FEE700BFB1
:1084F0001D0D0020501B0020FA01002084B02A4BE3
:108500009A6842F480729A609A6822F07F029A60B8
:108510001A6B0192019A42F04F020192019A22F4E1
:10852000074222F080020192019A42F40042019235
:10853000019A1A631C4B1B6B13F4004FFAD01A4AB2
:10854000136B0293029B43F04F030293029B43F48D
:1085500000430293029B136300238DF8033006E06F
:1085600000BF9DF803300133DBB28DF803309DF876
:108570000330DBB2132BF3D9EFF31083B3FA83F399
:108580005B09039372B6BFF35F8F0022074B1A702B
:10859000039B0121044A116123B1044B1970BFF3FD
:1085A0005F8F62B604B0704700400440FA010020BB
:1085B000034A0023136153619381024A1370704789
:1085C000381B0020220D002082B00522104B1A70AB
:1085D000104A136B0193019B43F04F030193019BDE
:1085E00043F020030193019B136300238DF80330B4
:1085F00006E000BF9DF803300133DBB28DF8033095
:108600009DF80330DBB2132BF3D902B0704700BFE3
:10861000220D00200040044082B00322104B1A704B
:10862000104A136B0193019B43F04F030193019B8D
:1086300043F010030193019B136300238DF8033073
:1086400006E000BF9DF803300133DBB28DF8033044
:108650009DF80330DBB2132BF3D902B0704700BF93
:10866000220D0020004004400422014B1A70704784
:10867000220D002008B5024B1B6903B1984708BDC5
:10868000381B002030B589B06A4B1B78032B29D0EA
:10869000694B9C89694B1B88E41AA4B2002C43D116
:1086A000674A11880B449BB21380634AD288934275
:1086B00003D0644B1B78002B2CD0634B9847634A44
:1086C000136B0393039B43F04F030393039B23F02C
:1086D00001030393039B13635C4B1B6B13F0010FAC
:1086E000FAD115E0594A136B0293029B43F04F03F2
:1086F0000293029B23F001030293029B1363534BEB
:108700001B6B13F0010FFAD1514B9847514B98470F
:1087100009B030BD484B5B6933B1984720B10022A6
:10872000464B1A80444B9C893F2C37D90022454B3D
:108730001A704024404B9A68404B1B881A44EFF350
:108740001083B3FA83F35B09079372B6BFF35F8FAD
:108750000021414B197007983C4B1B6B13F0020F23
:108760003ED028B101223C4B1A70BFF35F8F62B636
:108770000422304B1A70354A136B0493049B43F068
:108780004F030493049B23F001030493049B13639E
:108790002E4B1B6B13F0010FFAD1B9E70122294BC5
:1087A0001A70C7E7157829490D650133DBB201322C
:1087B00099B28C42F6D8214B1A8814441C80234A63
:1087C000136B0593059B43F04F030593059B43F003
:1087D00010030593059B136300238DF8073008E011
:1087E0000023E5E700BF9DF807300133DBB28DF8C9
:1087F00007309DF80730DBB2132BF3D9134A136B04
:108800000693069B43F04F030693069B23F0010358
:108810000693069B13630D4B1B6B13F0010FFAD1EC
:1088200000283FF475AF01220B4B1A70BFF35F8F26
:1088300062B66DE7220D0020381B00201E0D0020BF
:10884000200D00201C0D00206986400000400440DF
:1088500075864000B1854000FA01002010B586B051
:10886000654B1B78012B1ED0022B04D0042B02D0A9
:10887000624B984701E0624B9847624A136B009342
:10888000009B43F04F030093009B23F002030093EF
:10889000009B13635B4B1B6B13F0020FFAD15A4B17
:1088A000984706B010BD574B186BC0F30A40574BA2
:1088B0009B89574A14882218934201DA181B80B208
:1088C000524B9A682244002305E04E49096D11700D
:1088D0000133DBB2013299B28842F6D80444A4B223
:1088E0004B4B1C8040281BD0484B9C815B6913B1CB
:1088F0009847002832D0434A136B0293029B43F0FF
:108900004F030293029B23F002030293029B136323
:108910003C4B1B6B13F0020FFAD13E4B9847C0E75C
:108920003A4BDA883C4B1B8823449A42DCDD374BB8
:108930009B899C4227D0334A136B0593059B43F0D8
:108940004F030593059B23F002030593059B1363D7
:108950002C4B1B6B13F0020FFAD1A2E7274B984761
:10896000284A136B0193019B43F04F030193019B32
:1089700023F002030193019B1363224B1B6B13F043
:10898000020FFAD18DE7214B5B6953B19847E8B1EB
:1089900021491F4A0B88108803440B800023138051
:1089A000C9E7164B9847174A136B0393039B43F091
:1089B0004F030393039B23F002030393039B13636F
:1089C000104B1B6B13F0020FFAD16AE70B4B984761
:1089D0000C4A136B0493049B43F04F030493049BD2
:1089E00023F002030493049B1363064B1B6B13F0E9
:1089F000020FFAD155E700BF220D0020C9854000C3
:108A00007586400000400440B1854000381B0020BE
:108A10001E0D002019864000200D00200023042B8D
:108A200014D810B40A499A00D418A0000446084487
:108A3000407C214400F083026FF3C7124A74013373
:108A4000DBB2042BEED95DF8044B7047704700BFD2
:108A5000240D002038B5437C13F0100F16D00D46BE
:108A6000437C6FF30413437404687CB102F10C037C
:108A7000074951F8233013F4806F01D042F080028F
:108A80008168012D14BF00200120A04738BD00BF20
:108A90000040044010B500240BE023460134E4B24A
:108AA00003EB8303980022460121034B1844034B38
:108AB0009847042CF1D910BD240D0020558A4000A0
:108AC00010B500F00F02531E03EB83039C0001213D
:108AD00002482044024B984710BD00BF240D0020DF
:108AE000558A400030B482B00246441E3B4900F132
:108AF0000C0551F8253051F8251013F0020302D06F
:108B000001F0400151B9002B39D004EB84039900E6
:108B1000334B0B44597C6FF38301597404EB84038A
:108B200099002F4B0B445B7C13F00C0F32D12B4977
:108B300000F10C0551F825300093009B43F04F03E2
:108B40000093009B23F002030093009B41F8253023
:108B500002F10C03214951F8233013F0020FF7D131
:108B6000002838D0032836D004EB8404A2001C4B24
:108B700013445A7C012161F383025A742BE004EB05
:108B800084039900164B0B44597C012565F383013E
:108B90005974C3E711490C3051F820300193019BFF
:108BA00043F04F030193019B23F040030193019B8A
:108BB00041F8203002F10C03084951F8233013F03A
:108BC000400FF7D104EB8404A200054B13445A7CF8
:108BD0006FF383025A7402B030BC70470040044007
:108BE000240D0020F0B4461EB300334499002A4AF5
:108BF0000A445368D1680B449468641A128AC2F319
:108C00000902944209D31446002706EB8602950018
:108C1000214A2A442144D1601EE00127F5E71D784E
:108C20001E4A00F1140142F821505D7842F82150AB
:108C30009D7842F82150DD7842F821501D7942F8A4
:108C400021505D7942F821509D7942F82150DD791B
:108C500042F82150083C0833072CE0D807E01D7883
:108C600000F114020D4941F82250013C0133002C5F
:108C7000F5D1094BB1008819820010461A44527C84
:108C8000C2F3810203440132597C62F383015974B7
:108C90003846F0BC704700BF240D0020004004405F
:108CA00070B582B0441E04EB84039A00364B134423
:108CB0005B7CC3F3810328B1032801D0022202E0C8
:108CC000012200E001229A4254DDA20022449500D4
:108CD0002D4B2B44DA689B689A4205D32A4B2B44D0
:108CE0005B7C13F0400F48D00E460546274B984753
:108CF000FEB1274A0C3552F825300193019B43F011
:108D00004F030193019B43F010030193019B42F831
:108D1000253000238DF8033006E000BF9DF80330B6
:108D20000133DBB28DF803309DF80330DBB2132B37
:108D3000F3D940B104EB84039A00134B13445A7CDB
:108D40006FF386125A74A200224491000E4B0B441A
:108D5000DA689B689A4212D30B4B0B445B7C13F08E
:108D6000400F0ED1084B0B445A7C42F080025A74DB
:108D7000002000E0012002B070BD0020FBE70120D0
:108D8000F9E70120F7E700BF240D0020E58B400044
:108D9000004004402DE9F84305468446471EBB00C9
:108DA0003B449A002A4C1444A268E368A2EB030EE9
:108DB000B4F81080C8F3090862681A440C302549D9
:108DC00051F82060C6F30A4666B3B6450BD9B646DD
:108DD0004FF0000907EB870188001D4901447344E7
:108DE000CB6000210AE04FF00109F3E70CF1140316
:108DF000184850F823301370013101328E45F5D8F0
:108E00002846154B9847B9F1000F01D1B04507D955
:108E100005F10C030F4A52F8233013F0200F04D051
:108E2000BDE8F8834FF00009EAE70123AB40536146
:108E3000074ABB00D819810008461144C96802449A
:108E400091602A4600212046044B9847E8E700BF7E
:108E5000240D002000400440E58A4000558A40006F
:108E60002DE9F0418CB00124ADE12046B34B984789
:108E70000120FAE1BB003B449900B14A0A44537C0B
:108E8000C3F38101033161F383035374537C13F003
:108E9000200F00F0848013F00C0F3BD0A94A04F19E
:108EA0000C0152F821300193019B43F04F030193D1
:108EB000019B43F010030193019B42F821300023F2
:108EC0008DF8013006E000BF9DF801300133DBB2C0
:108ED0008DF801309DF80130DBB2132BF3D9994A9C
:108EE00006F10C0152F821300293029B43F04F032C
:108EF0000293029B23F001030293029B42F821306C
:108F000006F10C038F4A52F8233013F0010FF7D10A
:108F10000120AAE18B4A04F10C0152F8213003939D
:108F2000039B43F04F030393039B23F0010303933D
:108F3000039B42F8213006F10C03824A52F8233099
:108F400013F0010FF7D1114606F10C0352F823205C
:108F50000492049A42F04F020492049A42F02002D2
:108F60000492049A41F8232000238DF8023006E091
:108F700000BF9DF802300133DBB28DF802309DF85E
:108F80000230DBB2132BF3D907EB8707BA006C4B27
:108F900013445A7C6FF345125A74012065E113F0B3
:108FA000800F42D1BB003B449A00654B1344DA6802
:108FB0009B689A424CD307EB87039A00604B13449B
:108FC0005B7C13F04C0F43D1EFF31083B3FA83F3C0
:108FD0005B090B9372B6BFF35F8F00225A4B1A7076
:108FE0000B9B584A55612BB10122574B1A70BFF3A6
:108FF0005F8F62B6534A06F10C0152F82130059397
:10900000059B43F04F030593059B23F00103059354
:10901000059B42F8213006F10C034A4A52F82330EE
:1090200013F0010FF7D101201FE1BB003B449A0070
:10903000434B1344597C6FF3C7115974DA689A6033
:10904000404B5D61224600214046404B9847A9E7CE
:10905000002C4AD0032C48D007EB87039A00384BEA
:1090600013445B7C13F00C0F3FD0364A06F10C0121
:1090700052F821300693069B43F04F030693069B5C
:1090800043F010030693069B42F8213000238DF82D
:10909000033006E000BF9DF803300133DBB28DF8EA
:1090A00003309DF80330DBB2132BF3D9254A06F1C8
:1090B0000C0152F821300793079B43F04F030793AD
:1090C000079B23F001030793079B42F8213006F129
:1090D0000C031C4A52F8233013F0010FF7D1002182
:1090E00020461B4B98470120BFE0002C4AD0032CA0
:1090F00048D001212046164B984758B3114A06F133
:109100000C0152F821300893089B43F04F03089359
:10911000089B23F001030893089B42F8213006F1D5
:109120000C03084A52F8233013F0010FF7D1002145
:109130002046074B9847012097E000BF958D4000DF
:10914000240D002000400440FA010020558A400010
:10915000A18C40004749BB00D81982000A4492F80C
:1091600011E06FF3C71E82F811E0D2681F44BB0004
:1091700019448A60404B5D612246002140463F4BC6
:109180009847BBE7012120463D4B98473A4A06F1F4
:109190000C0152F821300993099B43F04F030993C6
:1091A000099B23F001030993099B42F8213006F142
:1091B0000C03314A52F8233013F0010FF7D101208C
:1091C00053E00134E4B2052C4ED82B4B9B69264664
:1091D0000125A5402B42F4D0671E07EB87029300C0
:1091E000244A02EB030804F10C03234A52F823300B
:1091F00013F0420F7FF439AE04F10C031E4A52F80B
:10920000233013F0010F7FF435AE04F10C031A4A3A
:1092100052F8233013F0080FD3D004F10C0152F8A8
:1092200021300A930A9B43F04F030A930A9B23F0D1
:1092300008030A930A9B42F8213006F10C030E4AF8
:1092400052F8233013F0080FF7D106F10C0352F84F
:10925000233003F4E063B3F5807F09D006F10C03FB
:1092600052F82330012000E000200CB0BDE8F0816E
:109270000120FAE7240D002000400440558A4000F8
:10928000A18C400000B587B0534B1B78E3B9534B1A
:109290001B6BC3F30A43082B3BD0504A136B01935B
:1092A000019B43F04F030193019B23F004030193BF
:1092B000019B1363494B1B6B13F0040FFAD1484B0E
:1092C000984707B05DF804FB464B9847464B9847D4
:1092D000DDE7424A116D454A99540133DBB2072B51
:1092E000F7D9434B9847B0B93C4A136B0293029BA2
:1092F00043F04F030293029B23F004030293029B6B
:109300001363364B1B6B13F0040FFAD1344B9847A1
:10931000D7E70023E3E7354B93F90030002B1EDB42
:109320002E4A136B0593059B43F04F030593059B52
:1093300023F004030593059B1363284B1B6B13F069
:10934000040FFAD1294BDB88002B42D00023294A95
:109350001380294A138001221F4B1A70B1E71F4A5C
:10936000136B0393039B43F04F030393039B43F05F
:1093700080030393039B136300238DF8033006E0FF
:1093800000BF9DF803300133DBB28DF803309DF848
:109390000330DBB2132BF3D9104A136B0493049BF5
:1093A00043F04F030493049B23F004030493049BB2
:1093B00013630A4B1B6B13F0040FFAD100230D4A01
:1093C00013800D4A13800222034B1A700B4B9847EF
:1093D00077E70B4B984774E7220D002000400440CC
:1093E000C985400075864000B1854000381B0020CB
:1093F00009824000200D00201E0D002085864000BF
:1094000019864000204BDB6913F0010F37D000B5FF
:1094100083B01D4B1B6B13F0040F24D11A4B1B6B35
:1094200013F0010F23D1184B1B6B13F0020F22D145
:10943000154B1B6B13F0080F23D0134A136B0193CA
:10944000019B43F04F030193019B23F00803019319
:10945000019B13630C4B1B6B13F0080FFAD1012017
:1094600003B05DF804FB094B98470120F8E7084B6F
:1094700098470120F4E7074B98470120F0E70020C8
:1094800070470020ECE700BF004004408592400098
:10949000858640005D88400010B54C4B984720B948
:1094A0004B4BDB6913F4807F10D03020494B984739
:1094B000474B9B6913F4006F04D0454BDB6913F4F1
:1094C000006F0AD1444B984770B110BD72B6BFF31C
:1094D0005F8F0022414B1A7010BD4FF400623C4B6D
:1094E0001A623F4B984710BD3E4B98470028ECD17D
:1094F000374B9B6913F4005F04D0354BDB6913F4E1
:10950000005F3DD1324B9B6913F4007F04D0304B98
:10951000DB6913F4007F33D12D4B9B6913F4806F0B
:1095200004D02B4BDB6913F4806F29D1284B9B6946
:1095300013F4807F04D0264BDB6913F4807F2FD196
:10954000234BDB6913F4805FBFD0214C4FF4805371
:109550002362254B9847254B9847636823F0010306
:109560006360636823F002036360214B9847214BDB
:1095700098474FF4807323614FF400632361A4E79D
:10958000134C4FF418532362636101201A4B984720
:109590004FF48073236223614FF40063236110BD95
:1095A0000B4B4FF480721A625A614FF400521A61E9
:1095B0004FF400721A614FF480621A6130200F4B31
:1095C000984700200C4B984710BD00BF9DA5400058
:1095D0000040044065A4400005944000FA010020CA
:1095E000D1814000618E4000958A4000F97F4000A3
:1095F000FD844000B185400059844000B9A440007A
:1096000010B582B0EFF31083B3FA83F35B090193D3
:1096100072B6BFF35F8F0022144B1A70019C0120B9
:10962000134B98473020134B9847134B5A6F22F433
:1096300080725A675A6F42F400725A674FF4807210
:109640001A614FF400521A614FF400721A614FF41C
:1096500080621A614FF400621A612CB10122034B3F
:109660001A70BFF35F8F62B602B010BDFA0100201E
:109670005984400065A440000040044030B583B0E8
:10968000EFF31083B3FA83F35B09009372B6BFF371
:109690005F8F0024204B1C70009D204B984730208A
:1096A0001F4B98471F4B98471F4B502283F830237E
:1096B0004FF480325A601D4B98474FF480201C4B6A
:1096C00098471C4B1C701C4B1B78FF2B22D0EFF3D0
:1096D0001083B3FA83F35B09019372B6BFF35F8F14
:1096E00000220D4B1A700199134A1378013313703D
:1096F00029B10122084B1A70BFF35F8F62B60F4B7E
:1097000098472DB10122044B1A70BFF35F8F62B6E8
:1097100003B030BDFEE700BFFA010020699E4000A3
:1097200065A4400051A0400000E100E01D8A400017
:1097300089A540001D0D0020501B0020019640000F
:109740000D4B5A6822F001025A609A6822F4807226
:109750009A60024670B1986820F07F0002F07F02A4
:10976000104398609A6842F480729A605A6842F096
:1097700001025A60704700BF00400440054B5B681F
:1097800013F0010F04D0034B986800F07F0070477E
:109790000020704700400440014B98609981704759
:1097A000381B0020F0B583B045B200F00F0005284B
:1097B00073D801F00306044600F10C033B4F57F841
:1097C000233013F4004F6BD1012E53D0031FDBB2B3
:1097D000012B54D94023934266DB461E06EB8607D5
:1097E000334B03EB870303F11007B3F810E062F388
:1097F000090EA3F810E05B7C03F07F036FF34513C1
:109800007B70002D3EDB294EB36A01228240134358
:10981000B362264B9B6A1A42FBD0244B9E6A26EA0F
:1098200002029A6200F10C0253F822300193019B6C
:1098300043F04F030193019B23F4074323F080037C
:109840000193002D23DB0A0202F4407242F400422D
:10985000019B1343019301990C30144B43F82010E2
:1098600004F10C03114951F8233032EA0303F7D114
:10987000012013E0B0B10328A8D100200EE04FF47E
:109880000073A8E77B786FF383037B70BBE70A0262
:1098900002F4407242F40442DAE7002003B0F0BD63
:1098A0000020FBE70020F9E70020F7E70040044034
:1098B000240D002000F00F03052B1ED810B582B038
:1098C00019460E4C0C3354F823200192019A42F0B1
:1098D0004F020192019A22F400420192019A44F847
:1098E000232001F10C03054A52F8233013F4004FF2
:1098F000F7D1034B984702B010BD704700400440B9
:10990000C18A400000F00F00431E052815D803EB64
:1099100083039A000A4B13445B7C13F0200F08D199
:109920000C30084B53F8203013F0280F03D00120DF
:10993000704701207047002070470020704700BF2B
:10994000240D00200040044010B485B044B200F063
:109950000F00052865D8421EEFF31083B3FA83F396
:109960005B09039372B6BFF35F8F0021314B19700F
:109970000399002C14DB304A00F10C0452F8243017
:109980000293029B43F04F030293029B43F0200398
:109990000293029B42F8243000238DF807302EE01A
:1099A00000F10C03244C54F8233013F0100F09D1AC
:1099B00002EB82039C00214B23445B7CC3F38103B5
:1099C000012BD8DD02EB820294001C4B23445A7C0D
:1099D00042F020025A74012303FA00F0164B18617A
:1099E00021B30120134B1870BFF35F8F62B619E0EB
:1099F00000BF9DF807300133DBB28DF807309DF8CA
:109A00000730DBB2132BF3D9012303FA00F00A4B22
:109A1000186169B10120074B1870BFF35F8F62B600
:109A200000E0002005B05DF8044B70470120F9E725
:109A30000120F7E7FA01002000400440240D002037
:109A400000F00F0005286CD830B583B00246441EE4
:109A500004EB84039900354B0B44597C6FF345119B
:109A6000597400F10C03324951F8233013F0200FE0
:109A700059D000F10C0551F825300093009B43F0BC
:109A80004F030093009B23F020030093009B41F8B9
:109A9000253002F10C03264951F8233013F0200F32
:109AA000F7D10D468B6A012181400B43AB62204BFD
:109AB0009B6A1942FBD01E4B9D6A25EA01019962FF
:109AC0000C3053F820100191019941F04F010191A0
:109AD000019921F008010191019943F8201002F148
:109AE0000C03134951F8233013F0080FF7D104EB9E
:109AF00084039A000D4B13445B7C13F0100F01D1CB
:109B0000012011E00949A200101983000B44587C80
:109B10006FF3041058741444A300CB5898470120E5
:109B200002E000207047012003B030BD240D00206A
:109B300000400440F0B583B000F00F04052C00F2A3
:109B4000A28047B2651E04F10C00554E56F8200065
:109B500010F4004F00F09A8005EB8500514E06EBA3
:109B60008000407C10F0200F40F0928004F10C0047
:109B70004B4E56F8200010F0200F40F08B80EFF392
:109B80001080B0FA80F04009009072B6BFF35F8F8A
:109B9000002645480670DDF800E005EB8500414EE3
:109BA00006EB8000407C10F0100F0AD0BEF1000FD1
:109BB00072D001223C4B1A70BFF35F8F62B6002057
:109BC00062E005EB8500374E06EB8000467C46F0F0
:109BD00010064674BEF1000F05D00126324806700B
:109BE000BFF35F8F62B6DFF8BCE005EB8500800055
:109BF0000EEB00067260B3600022F260089A4EF825
:109C0000002011B95BBB012000E00120254AA9001A
:109C10004B1902EB83035B7C60F386130D4402EB6C
:109C200085026FF3C7135374EFF31083B3FA83F312
:109C30005B09019372B6BFF35F8F00221A4B1A7053
:109C4000019D0123A340164A1361002F09DB2DB3A8
:109C50000120154B1870BFF35F8F62B614E000202F
:109C6000D4E704F10C0352F8233013F0110FEED1B6
:109C7000012120460D4B98470028E8D000212046BE
:109C80000A4B9847E3E7002003B0F0BD0020FBE754
:109C90000020F9E70020F7E70020F5E70120F3E7CF
:109CA00000400440240D0020FA010020A18C400057
:109CB00070B586B000F00F04052C00F2C98042B2E6
:109CC000EFF31083B3FA83F35B09059372B6BFF326
:109CD0005F8F00215F4B1970059B26460125A5402B
:109CE0005D494D612BB101215A4B1970BFF35F8F54
:109CF00062B6002A80F2948004F10C03564A52F8AE
:109D0000233013F0100F64D0002C49D0032C47D01F
:109D100004F10C0152F821300193019B43F04F03F1
:109D20000193019B23F010030193019B42F8213022
:109D300006F10C03484A52F8233013F0100FF7D104
:109D400006F10C03444A52F8233013F0100FF7D1F8
:109D500004F10C0152F821300293029B43F04F03AF
:109D60000293029B43F010030293029B42F82130BE
:109D700000238DF8033006E000BF9DF80330013367
:109D8000DBB28DF803309DF80330DBB2132BF3D92F
:109D900006F10C03304A52F8233013F0100FF7D0BD
:109DA0002D4A04F10C0152F821300393039B43F038
:109DB0004F030393039B23F010030393039B42F889
:109DC000213006F10C03244A52F8233013F0100F0F
:109DD000F7D1214A04F10C0152F821300493049B7D
:109DE00043F04F030493049B23F001030493049B6B
:109DF00042F8213006F10C03174A52F8233013F0D1
:109E0000010FF7D1621E02EB82029100134B0B444B
:109E10005A7C6FF383025A740AE02046104B98472D
:109E200006F10C030C4A52F8233013F0420FF4D120
:109E3000094A936A2B439362074B9B6A1D42FBD0EE
:109E4000054A936A23EA050595622046054B984723
:109E500006B070BDFA01002000400440240D00202F
:109E6000E58A4000C18A4000064BD3F8142122F451
:109E70004062C3F81421D3F8202142F00102C3F854
:109E80002021704700020E400B4619B1096801609D
:109E90005B6843601AB1136803615368436170479C
:109EA00021F0FE01C905C90D0162704710B51E4BB6
:109EB00053F820402268536A13F0805F11D00223C8
:109EC000C2F8203123684FF0FF32DA610023237596
:109ED000236913F0010F26D0636823B32046984707
:109EE00010BD13F0006F13D00223C2F82031236895
:109EF0004FF00062DA61236913F0020F03D0A36808
:109F00000BB12046984723680122C3F8202110BDD9
:109F100013F0007F07D0236913F0040F03D0E36828
:109F20000BB12046984710BD880D002008B50020D1
:109F3000014B984708BD00BFAD9E400008B5012009
:109F4000014B984708BD00BFAD9E400070B5054667
:109F50000E461446016001230B60214B99422BD021
:109F60000D20204B9847204B1D6023781B0203F4E3
:109F7000FE43736063782BBB0022A3780BB142F0E1
:109F80000402E3780BB142F0080223790BB142F0EE
:109F9000100263791B0203F47063A179090389B28B
:109FA0000B431343B3652389C3F30E03628943EA6A
:109FB0000243F36500230CE012200A4B98470A4B3A
:109FC0005D60D2E70222D8E705EB830200215160F1
:109FD0000133022BF8D900202861287570BD00BF1D
:109FE0000000034065A44000880D002012F0100F0F
:109FF00012D0C0F8B01012F0200F07D0C0F8D41063
:10A0000012F0400F05D0C0F8C0107047C0F8D01053
:10A01000F6E7C0F8C4107047C0F8B4107047016488
:10A02000704741647047C06C7047806C704740094E
:10A0300000F5001000F207704002704740090B3035
:10A04000704700F01F00012303FA00F07047000082
:10A0500008B500200A4B98470A4B98470028FBD0C8
:10A06000094B9847094A0A4BDA620A4B984700287D
:10A07000FBD00020084B9847084B984708BD00BF0D
:10A08000E1A3400005A4400049A44000013FB805F9
:10A0900000040E4055A4400069A540007DA5400085
:10A0A00010B5A2B01848194B98470020184B984794
:10A0B000184B98470028FBD0174B9847174A184B66
:10A0C0009A62184B98470028FBD00020164B9847FF
:10A0D000164B984716480D4B9847164B1A68164B67
:10A0E0001344164A934201D922B010BD2023009395
:10A0F00002AB0F220E211248124CA047BDF84810A7
:10A100001148124B9847EFE7000E2707D5A84000EB
:10A11000E1A3400005A440002DA44000013FB70B7F
:10A1200000040E4039A440008DA34000E1A7400088
:10A130000000DC05FC010020C0D3BDF980C3C901CB
:10A14000000A0E400100002010140E40ADA5400092
:10A1500070B50D461446064658B14FF0FF360AE07A
:10A16000064B1868064B1B6829469847013501368F
:10A17000013C002CF4DC304670BD00BF601B0020A9
:10A18000581B002070B5013802280FD8144600254E
:10A190008CB10A4B18684E1C094B1B68097898470C
:10A1A000002806DB0135013C3146F1E74FF0FF3571
:10A1B00001E04FF0FF35284670BD00BF601B002056
:10A1C0005C1B0020A1F10E03012B02D84FF0FF30E1
:10A1D000704710B582B0EFF31083B3FA83F35B09D5
:10A1E000019372B6BFF35F8F00240B4B1C70019C70
:10A1F000120222F07F4222F0FF02C9B2114341F065
:10A20000B441064B98472CB10122034B1A70BFF39F
:10A210005F8F62B602B010BDFA0100206900002015
:10A220004C4B1B78FF2B31D000B583B0EFF310837C
:10A23000B3FA83F35B09019372B6BFF35F8F002219
:10A24000454B1A700199434A13780133137029B1B1
:10A250000122414B1A70BFF35F8F62B63F4A9042B2
:10A2600015D03F4A904220D03E4A90422BD03E4AE1
:10A27000904236D03D4A904241D03D4A90424CD027
:10A280003C4A904257D003B05DF804FBFEE716202D
:10A29000394B98470720394B984700210720384B06
:10A2A00098470720374B9847EDE71520324B9847E2
:10A2B0000720324B984700210720314B9847072051
:10A2C000304B9847DFE714202B4B984707202B4B48
:10A2D0009847002107202A4B98470720294B984789
:10A2E000D1E71320244B98470620244B98470021A0
:10A2F0000620234B98470620224B9847C3E70E20A1
:10A300001D4B984706201D4B9847002106201C4BEB
:10A31000984706201B4B9847B5E70920164B9847EE
:10A320000620164B984700210620154B984706201B
:10A33000144B9847A7E708200F4B984706200F4B70
:10A340009847002106200E4B984706200D4B984752
:10A3500099E700BF501B0020FA01002000000440D4
:10A360000080004000C001400080014000400240E9
:10A370000000024000C0004065A4400055A5400018
:10A380000DA5400041A5400001607047134A136BC2
:10A3900023F07003184310634FF400630F4A926E6A
:10A3A00012F0080F02D1A3B1013BF7E70B4A136B80
:10A3B00023F0030343F0020313634FF40063074ADF
:10A3C000926E12F0080F02D12BB1013BF7E700208B
:10A3D0007047012070470120704700BF00040E4005
:10A3E000012803D0054A064B1A607047044A936857
:10A3F00043F0254343F480139360F3E7080000A57E
:10A4000010140E40074B5B6913F0800F06D0064B0B
:10A410009B6E13F0800F03D100207047002070471F
:10A420000120704710140E4000040E400022014B22
:10A430009A62704700040E40024B986E00F00200D2
:10A44000704700BF00040E400022014BDA627047E3
:10A4500000040E40024B986E00F00400704700BFED
:10A4600000040E4032281ED81F280CD8114B9A69C0
:10A4700001238340934318D0012303FA00F00D4BCE
:10A4800018610020704720380A4BD3F808210123B7
:10A49000834093430BD0012303FA00F0054BC3F82C
:10A4A0000001002070470120704700207047002005
:10A4B000704700BF00040E40322822D81F280ED853
:10A4C000114B9A6901238340934301D000207047C8
:10A4D000012303FA00F00C4B58610020704720382C
:10A4E000094BD3F8082101238340934301D0002076
:10A4F0007047012303FA00F0034BC3F80401002066
:10A5000070470120704700BF00040E4041F0040175
:10A5100000F11002094B43F822104FF40062074B80
:10A52000996E4FF480738340194202D11AB1013AF7
:10A53000F5E7002070470120704700BF00040E407F
:10A540004FF4807303FA00F0014B1860704700BFAE
:10A5500000040E404FF4807303FA00F0014B586082
:10A56000704700BF00040E40000200F4706040F02D
:10A570000100014B9863704700040E408022014B9C
:10A580001A60704700040E40C0F31200024B1A6FAD
:10A5900010431867704700BF00040E40024B187844
:10A5A00080F00100704700BF900D0020C36923F4C4
:10A5B000F053490201F4F051194341F0B44141F420
:10A5C0008071C161704730B4B2EB011F17D3102402
:10A5D00001FB04F14B0803EBC202B2FBF1F2D3081A
:10A5E0005D1E4FF6FE718D4210D8082C09D0120462
:10A5F00002F4E0221A430262002030BC70470824B3
:10A60000E6E7416841F400214160F0E70120F4E70A
:10A610004023036070478823036070471023036062
:10A6200070472423036070474FF4807303607047C2
:10A630004FF4002303607047436913F0020F04D006
:10A64000C1F30801C16100207047012070474369D0
:10A6500013F0020FFBD0C1F30801C1610020704765
:10A66000436913F0010F05D08369C3F308030B603E
:10A670000020704701207047014BC0F8E43070475C
:10A680000041535510B50446094B984700236360B9
:10A690006362A3622046074B98472046064B9847C3
:10A6A0002046064B98472046054B984710BD00BFF3
:10A6B00079A6400017A6400023A6400029A6400026
:10A6C00031A6400070B505460C461646104B98471B
:10A6D0000022104B1A60B4B13246216828460E4B56
:10A6E0009847024688B96368A1680B4321690B4308
:10A6F000E1680B430749086803430B6069680B4333
:10A700006B60104670BD0122FBE70122F9E700BF34
:10A7100085A64000940D0020C7A54000FEE700007C
:10A7200000B583B0234B244A9A4209D0214B224AD8
:10A7300003E0116819600433043220498B42F8D3D6
:10A740001F4B02E000221A6004331E4A9342F9D3E1
:10A750001D4A22F07F011D4B9960EFF31083B3FA7D
:10A7600083F35B09019372B6BFF35F8F0021184B2F
:10A770001970019817490B6843F470030B60BFF31D
:10A780004F8FBFF36F8F28B10121114B1970BFF3A9
:10A790005F8F62B602F16042B2F5203F04D20B4AED
:10A7A000936843F0005393600B4B98470B4B9847CB
:10A7B000FEE700BF0000002090064100B80B00201B
:10A7C000B80B0020B41B00200040400000ED00E06A
:10A7D000FA01002088ED00E0EDD04000EDC040001F
:10A7E000344B1B6B03F00303012B20D083B1022BEE
:10A7F00039D0304B1B6B03F07003702B51D02D4BB5
:10A800001A6BC2F302122C490B68D3400B607047DD
:10A810002A4B5B6913F0800F04D04FF40042264BA3
:10A820001A60E6E74FF4FA42234B1A60E1E7214B46
:10A830001B6A13F0807F03D0214A1F4B1A60D8E7B0
:10A84000204A1D4B1A601B4B1B6A03F07003102B30
:10A8500005D0202BCDD11C4A174B1A60C9E71B4AE3
:10A86000154B1A60C5E7154B5B6913F0800F13D0C9
:10A870004FF40042104B1A600E4B1B6B03F00303A6
:10A88000022BB6D10B4B9A6AC2F30C420A490B68F1
:10A8900002FB03330B60ACE74FF4FA42064B1A603D
:10A8A000EAE7054A13680A49A1FB03135B08136032
:10A8B000704700BF00040E40FC01002010140E4041
:10A8C000001BB70000127A0000366E010024F4006D
:10A8D000ABAAAAAA144B98420FD9144B984211D98B
:10A8E000134B984212D9134B984213D9124B9842EA
:10A8F00014D9124A124B1A6070474FF08062104B05
:10A900001A6070470F4A0E4B1A6070470E4A0C4B84
:10A910001A6070470D4A0A4B1A6070474FF00422C4
:10A92000074B1A60704700BFFF2C3101FF596202CC
:10A93000FF869303FFB3C404FFE0F50500050004A0
:10A94000000A0E400001000400020004000300049D
:10A950000A4B1B6853B1094B1B681A1808499142EE
:10A9600008DB1046054A106018467047054A034B3D
:10A970001A60F0E74FF0FF30704700BF980D0020DD
:10A98000FC7F0220B84B00204FF0FF3070474FF49F
:10A9900000534B6000207047012070470020704733
:10A9A00000F1080343604FF0FF328260C36003612F
:10A9B00000230360704700230361704743684B60C6
:10A9C0009A688A609A6851609960086103680133E7
:10A9D0000360704730B40D68B5F1FF3F02D000F15D
:10A9E000080202E0026904E01A4653681C68A542A6
:10A9F000FAD253684B6099608A60516008610368BD
:10AA00000133036030BC704703694268816891601C
:10AA10008268416851605A68904206D00022026103
:10AA20001A68013A1A601868704782685A60F5E738
:10AA300082B0002301934FF0500383F31188BFF3DA
:10AA40006F8FBFF34F8F019B002BFCD002B070477C
:10AA500008480068006880F308884FF0000080F321
:10AA6000148862B661B6BFF34F8FBFF36F8F00DFFC
:10AA700000BF000008ED00E0DFF80C00016841F4C1
:10AA8000700101607047000088ED00E04FF08073B6
:10AA900040F8043C21F0010140F8081C054B40F847
:10AAA0000C3C40F8202C6FF0020340F8243C443862
:10AAB000704700BF31AA4000000000000000000005
:10AAC000074B19680868B0E8F04F80F30988BFF3B6
:10AAD0006F8F4FF0000080F311887047AFF3008054
:10AAE0009C0D00204FF0500383F31188BFF36F8F4C
:10AAF000BFF34F8F024A136801331360704700BFE2
:10AB000000020020034A1368013B13600BB983F372
:10AB100011887047000200200000000000000000C3
:10AB2000EFF30980BFF36F8F154B1A681EF0100FFB
:10AB300008BF20ED108A20E9F04F10602DE90900D0
:10AB40004FF0500080F31188BFF34F8FBFF36F8F2A
:10AB500000F03CFE4FF0000080F3118809BC19683A
:10AB60000868B0E8F04F1EF0100F08BFB0EC108A74
:10AB700080F30988BFF36F8F704700BFAFF3008089
:10AB80009C0D002008B54FF0500383F31188BFF3EC
:10AB90006F8FBFF34F8F054B984718B14FF080521E
:10ABA000034B1A60002383F3118808BD49B54000A8
:10ABB00004ED00E0054B00221A6005490A600549D2
:10ABC000054A116007221A60704700BF10E000E0DC
:10ABD00018E000E0FF7F010014E000E010B50E4B2C
:10ABE0001A6842F470021A601A6842F070421A60E1
:10ABF0000A4B984700240A4B1C600A4B98470A4AA4
:10AC0000136843F040431360084B9847084B98473C
:10AC1000084B9847204610BD20ED00E0B5AB400042
:10AC20000002002079AA400034EF00E051AA400061
:10AC3000CDB7400031AA400010B50446044B9847F8
:10AC40002046044B98470446034B9847204610BDC6
:10AC500039B5400065D140003DB6400048B110B55F
:10AC60000446044B98472046034B9847034B9847AC
:10AC700010BD704739B5400075D140003DB6400069
:10AC8000436A23B1036B1868C0F1050070470020C8
:10AC90007047000010B50446064B9847A26BE36B63
:10ACA0009A4204D00024044B9847204610BD01244A
:10ACB000F9E700BFE5AA400005AB400010B5044627
:10ACC000054B9847A36B23B10024044B98472046BB
:10ACD00010BD0124F9E700BFE5AA400005AB400024
:10ACE00070B504461646856B026C5AB903681BB1F1
:10ACF00000200135A56370BD4068174B98470023BD
:10AD00006360F6E76EB98068144B9847226CA368BD
:10AD10001344A3606268934219D32368A3600020A0
:10AD2000E7E7C0680D4B9847226C5242E368134432
:10AD3000E36021688B4202D263681A44E260022E0B
:10AD400001D00020D5E725B1013D0020D1E700204A
:10AD5000CFE70020CDE700BF81BA400091D7400087
:10AD600038B505461A4B984795F8454064B201E05E
:10AD7000013C64B2002C0ADD6B6A43B105F124008A
:10AD8000144B98470028F3D0134B9847F0E7FF2364
:10AD900085F84530114B98470D4B984795F844403E
:10ADA00064B201E0013C64B2002C0ADD2B6943B1BE
:10ADB00005F11000074B98470028F3D0064B984741
:10ADC000F0E7FF2385F84430044B984738BD00BFB7
:10ADD000E5AA4000A5B84000A1B9400005AB40007D
:10ADE00038B504460D46144B98472168E26B236C36
:10ADF00003FB021060600020A063A160013A02FB27
:10AE00000313E360FF2384F8443084F8453055B9D8
:10AE100023691BB9094B9847012038BD04F1100084
:10AE2000074B9847F6E704F11000064DA84704F1D8
:10AE30002400A847EEE700BFE5AA400005AB4000AC
:10AE4000A5B84000A1A9400038B51D46049C0B469A
:10AE500049B12260E063236401212046034B9847F7
:10AE600084F84C5038BD2460F4E700BFE1AD4000E9
:10AE7000F0B583B0054617460E4689B100FB01F0D8
:10AE80005030084B9847044638B100903B4600F1DB
:10AE9000500231462846044DA847204603B0F0BD75
:10AEA0000020EDE739AC400049AE4000F0B585B078
:10AEB00004460F4601921E46002526E032463946DA
:10AEC0002046354B9847636A23B9344B9847012095
:10AED00005B0F0BD04F12400314B9847F5E72F4B46
:10AEE00098470020F4E702A82E4B9847012519E067
:10AEF000002384F8443021E0002384F8453023E027
:10AF00002046294B9847294B9847294B9847A26BD5
:10AF1000E36B9A42D2D3022ED0D0019B002BDED01D
:10AF2000002DE0D01D4B9847224B9847204B984767
:10AF300094F844305BB2B3F1FF3FD9D094F8453078
:10AF40005BB2B3F1FF3FD7D0144B984701A902A8D9
:10AF5000194B9847C8B92046184B98470028CFD0BE
:10AF6000019904F11000164B984720460E4B984764
:10AF70000E4B98470028C8D14FF08052114B1A60F1
:10AF8000BFF34F8FBFF36F8FBFE72046064B984745
:10AF9000064B984700209BE7E1AC400005AB400022
:10AFA000A5B8400025B9400061AD40003DB6400065
:10AFB000E5AA400039B540003DB9400095AC4000DD
:10AFC00081B8400004ED00E048B110B500214160B7
:10AFD0000160C1600B460A46014CA04710BD704796
:10AFE000ADAE400010B5024600210120034B98474A
:10AFF0000446034B9847204610BD00BF71AE400089
:10B00000C9AF400070B584B00446019100263546B2
:10B010003EE0013BA36323683BB123694BB9444B3A
:10B0200098470126304604B070BD424B9847606097
:10B03000F3E704F11000404B9847F0E73C4B98478A
:10B040000026EFE702A83D4B984701252AE00023A0
:10B0500084F8443032E0002384F8453034E0384B43
:10B0600098476068374B98470646314B98473BE016
:10B070002046354B9847354B984709E02046324BE0
:10B080009847324B98472046314B9847002840D18B
:10B090002B4B9847A36B002BBBD1019B002BCDD032
:10B0A000002DCFD0224B98472A4B9847244B9847E6
:10B0B00094F844305BB2B3F1FF3FC8D094F8453008
:10B0C0005BB2B3F1FF3FC6D0194B984701A902A864
:10B0D000214B98470028D1D120461D4B9847002886
:10B0E000C6D02368002BBAD0019904F124001B4B71
:10B0F00098472046144B9847144B98470028C7D1CF
:10B100004FF08052164B1A60BFF34F8FBFF36F8F13
:10B11000BEE7002E86D00A4B98472046114B984731
:10B1200001466068104B9847014B9847002679E725
:10B1300005AB4000A9BB4000A5B8400025B94000C0
:10B14000E5AA4000B9B9400061AD40003DB64000FD
:10B15000BDAC400039B540003DB9400081B8400069
:10B1600004ED00E081AC400009BB4000F0B503688D
:10B170004BB343685B68436000F10807BB4204D0EF
:10B180004368D3F80CE0002609E05B684360F7E70A
:10B190005B68436008E02E46B6B9AE4514D04368FC
:10B1A0005B6843609F42F3D04368DD6800230F2B48
:10B1B000F2D8EA1892F83420CC5CA242ECD1002AF2
:10B1C000E9D00133F3E700263046F0BD0A4B1B6897
:10B1D0001B684BB901234BB9074B1B68DB68DB6865
:10B1E0005A68064B1A6070470023F4E74FF0FF32AD
:10B1F000024B1A60704700BFA00D00204C0E0020CB
:10B200002DE9F84F81460D4617469A460A9EDDF80D
:10B210002C800C9C9200A521206B1D4B9847236B22
:10B2200007F18042013A03EB820727F0070700236A
:10B230000F2B07D8E95CE21882F83410EA5C0AB1F7
:10B240000133F5E7002384F84330042E00D90426A7
:10B25000E662E66400252565201DDFF83CB0D8478E
:10B2600004F11800D8472461C6F10506A66164629E
:10B27000656584F85850524649463846054B98470C
:10B280002060B8F1000F01D0C8F80040BDE8F88F89
:10B290008DD940008DAA4000B7A9400070B50024A8
:10B2A00007E004EB840293000B4818440B4B9847CB
:10B2B0000134042CF5D90A4E3046084CA047094DFC
:10B2C0002846A0470848A0470848A047084B1E60EA
:10B2D000084B1D6070BD00BFA80D0020A1A9400053
:10B2E000200E0020340E0020540E00206C0E002092
:10B2F000A00D0020A40D002010B504461C4B98475B
:10B300001C4A1368013313601B4B1B68002B26D0AB
:10B310001A4B1B683BB9184B1B68DA6AE36A9A42FE
:10B3200001D8154B1C60164A13680133136063641F
:10B33000E36A01229A401349086802430A6003EB5A
:10B3400083039A00211D10481044104B9847104B5E
:10B3500098470A4B1B680BB1074B1B6810BD064B87
:10B360001C601368012BDED10A4B9847DBE700BF56
:10B37000E5AA40000C0E00209C0D0020680E002065
:10B38000180E00201C0E0020A80D0020BDA94000B2
:10B3900005AB40009DB2400070B504460E461D4B03
:10B3A0001D681D4B186804301C4B984750B91A4B48
:10B3B0001B68DA6A012303FA02F219490B6823EACF
:10B3C00002030B60B4F1FF3F13D02C44124B1B68F7
:10B3D0005C60A54216D8134B18680F4B19680431EE
:10B3E000114B9847114B1B689C4201D20F4B1C60BC
:10B3F00070BD002EE9D0084B196804310C480D4B84
:10B40000984770BD0C4B1868034B19680431064B04
:10B41000984770BD800E00209C0D002009AA4000B6
:10B420001C0E0020A00D0020D5A940004C0E0020CD
:10B430006C0E0020BDA94000A40D002008B54FF0FF
:10B440008052044B1A60BFF34F8FBFF36F8F024BD4
:10B450009847F4E704ED00E0E9C040002DE9F0432F
:10B4600085B006460F46154698469000144B9847FF
:10B4700000B381465C20124B98470446B0B1C0F837
:10B480003090CCB10023039302940D9B01930C9B4D
:10B49000009343462A46394630460A4DA84720467F
:10B4A000094B9847012005B0BDE8F0834846074B9B
:10B4B0009847E6E70024E4E74FF0FF30F3E700BFEA
:10B4C00039AC400001B24000F9B240005DAC400030
:10B4D00010B582B0104B01930023009346220F4910
:10B4E0000F48104CA047012801D002B010BD4FF00A
:10B4F000500383F31188BFF36F8FBFF34F8F4FF06B
:10B50000FF32094B1A600122084B1A600022084BD7
:10B510001A60084B9847E8E7480E002030044100C5
:10B520003DB440005DB440004C0E0020680E002089
:10B53000800E0020DDAB4000024A13680133136027
:10B54000704700BF140E002070B52F4B1B68002BF6
:10B5500052D12E4B1E6801361E604EB12C4B1B681B
:10B560009E422FD22B4B1B68002B42D0002070BD77
:10B57000294A1168294B186810601960284A136815
:10B5800001331360274B9847E8E7012320E04FF091
:10B59000FF321F4B1A60E5E71D4A1360E2E704F132
:10B5A0001800214B9847E36A01229A401F49086816
:10B5B00002430A6003EB83039A0029461C481044A7
:10B5C0001C4B9847144B1B681B68002BDDD00023D5
:10B5D000002BDCD1104B1B68DB68DC6863689E4283
:10B5E000DAD3251D2846104B9847A36A002BD6D1E5
:10B5F000D9E7114B9847B9E7064A1368013313603E
:10B600000D4B9847B2E700BF140E0020800E0020BB
:10B610004C0E0020100E0020A00D0020A40D0020D4
:10B62000500E0020CDB1400009AA40001C0E0020A1
:10B63000A80D0020BDA94000EBC0400070B5274B0D
:10B640009847274B1A68013A1A601B68002B32D1C1
:10B65000244B1B68002B2ED00024234B1B6813B3F4
:10B66000214BDB68DC6804F11800204EB047251D33
:10B670002846B047E36A01229A401D490868024300
:10B680000A6003EB83039A0029461A4810441A4BB8
:10B690009847E26A194B1B68DB6A9A42DDD30122A4
:10B6A000174B1A60D9E70CB1164B9847164B1C681C
:10B6B0003CB9134B1B68154B9847002070BD013CEB
:10B6C00007D0134B98470028F9D001220C4B1A6081
:10B6D000F5E700220C4B1A60EBE700BFE5AA40003B
:10B6E000140E00200C0E0020540E002009AA400069
:10B6F0001C0E0020A80D0020BDA940009C0D0020BC
:10B70000840E0020CDB14000100E002005AB40009B
:10B7100049B5400010B550B9002038B94FF08052FB
:10B72000084B1A60BFF34F8FBFF36F8F10BD0446F5
:10B73000054B984700212046044B9847044B9847F7
:10B74000EBE700BF04ED00E039B5400099B34000DD
:10B750003DB6400070B50646154B98470524013CA0
:10B7600004EB84029300314612481844124B984768
:10B77000054608B9002CF2D12DB15DB18DB10F4B4A
:10B780009847284670BD0E4B186831460A4B9847BB
:10B790000546F2E70B4B18683146074B98470546BC
:10B7A000ECE731460848044B98470546E7E700BFF9
:10B7B00039B54000A80D00206DB140003DB64000F5
:10B7C000A00D0020A40D00206C0E0020264B1B684D
:10B7D000002B2FD110B50022244B1A60244B1B687C
:10B7E0001B6B1A68B2F1A53F28D0214B1868196865
:10B7F0003431204B9847204B1B68B3FA83F3DBB2FC
:10B80000C3F11F031D489A00D418A10001444C68DD
:10B8100064684C601A4491000831084484421AD08C
:10B8200003EB83039A00154B13445B68DA68104BF3
:10B830001A6010BD01220D4B1A6070475A68B2F1B0
:10B84000A53FD2D19A68B2F1A53FCED1DB68B3F162
:10B85000A53FCAD1CFE7606803EB83029100074A96
:10B860000A445060DCE700BF140E0020840E002064
:10B870009C0D0020D1C040001C0E0020A80D00200F
:10B8800010B50C46044B19681831044B9847012138
:10B890002046034B984710BD9C0D0020D5A94000C1
:10B8A00099B3400038B5C368DC6804F11805284630
:10B8B000144B9847144B1B68E3B9251D2846114BC0
:10B8C0009847E36A01229A401049086802430A60D7
:10B8D00003EB83039A0029460D4810440D4B98470B
:10B8E000E26A0D4B1B68DB6A9A4208D901200B4BB8
:10B8F000186038BD29460A48064B9847F0E70020F3
:10B9000038BD00BF09AA4000140E00201C0E002004
:10B91000A80D0020BDA940009C0D0020840E002031
:10B92000540E0020034B1B680360034B1B684360ED
:10B93000704700BF500E0020800E0020F8B504466E
:10B940000D46124B9847124B19686268881A2B688B
:10B95000B3F1FF3F16D027680E4E3668B74201D0CC
:10B96000914211D2984206D300232B6001240A4B46
:10B9700098472046F8BD1B1A2B602046074B984776
:10B980000024F4E70024F2E70124F0E7E5AA4000F0
:10B99000800E0020500E002005AB400025B940006D
:10B9A0000122014B1A607047840E0020014B186879
:10B9B000704700BF9C0D0020002854D038B50446C5
:10B9C000C26A2A490968C96A8A4242D28169002941
:10B9D00005DB26490968C96AC1F105018161606911
:10B9E00002EB82029100224A0A44904207D00022D0
:10B9F0003AB91E4A1268D26AE262012038BD0122B9
:10BA0000F6E7251D28461B4B984768B9E36A03EB08
:10BA100083018A0016498A5832B901229A40164990
:10BA20000B6823EA02030B60104B1B68DB6AE362BE
:10BA3000012404FA03F21049086802430A6003EB88
:10BA400083039A0029460A4810440C4B9847204625
:10BA500038BDC26C054B1B68DB6A9A4201D20120DB
:10BA600038BD002038BD0020704700BF9C0D00206D
:10BA7000A80D002009AA40001C0E0020BDA940000E
:10BA8000002834D038B50446026D013A0265C06A18
:10BA9000E16C88422DD00AB1002038BD251D284612
:10BAA000154B984768B9E36A03EB83018A00134991
:10BAB0008A5832B901229A4011490B6823EA0203DD
:10BAC0000B60E36CE362C3F10502A261012404FA96
:10BAD00003F20B49086802430A6003EB83039A00F0
:10BAE000294606481044074B9847204638BD002099
:10BAF0007047002038BD00BF09AA4000A80D0020F3
:10BB00001C0E0020BDA94000002843D038B50446D3
:10BB1000C26C8A4200D20A46E16A8A4202D0206D93
:10BB2000012800D038BDE262A069002802DBC2F122
:10BB30000502A261636901EB81018800164A024493
:10BB4000934225D00022002AECD0251D2846134B15
:10BB5000984768B9E36A03EB83018A000E498A5863
:10BB600032B901229A400E490B6823EA02030B60A6
:10BB7000E36A01229A400A49086802430A6003EB1B
:10BB800083039A00294604481044064B9847C9E7A6
:10BB90000122D8E7704700BFA80D002009AA400085
:10BBA0001C0E0020BDA94000054B1B6823B1044BAF
:10BBB0001A68136D01331365014B1868704700BF95
:10BBC0009C0D002038B505460C461A4B98471A4B79
:10BBD0001B685B6D2BB9184B1B68012283F858203A
:10BBE000ACB9164B9847134B9847134B1B685C6DC9
:10BBF00024B1CDB9104B1B68621E5A650E4B1B68F1
:10BC0000002283F858200D4B9847204638BD114636
:10BC100020460B4B98474FF080520A4B1A60BFF3F7
:10BC20004F8FBFF36F8FDCE7034B1B6800225A6511
:10BC3000E4E700BFE5AA40009C0D002005AB4000F2
:10BC400099B3400004ED00E0F8B5EFF311854FF033
:10BC5000500484F31188BFF36F8FBFF34F8F0BB184
:10BC6000446D1C6090F85830DBB2022480F85840D4
:10BC7000013A032A1AD8DFE802F0020C1114426DCF
:10BC8000114341650126012B14D085F311883046FC
:10BC9000F8BD426D013242650126F4E74165012697
:10BCA000F1E7022B04D041650126ECE70126EAE723
:10BCB0000026E8E70446164B1B68F3B9071D384613
:10BCC000144B9847E36A01229A40134908680243DB
:10BCD0000A6003EB83039A00394610481044104B66
:10BCE0009847E26A0F4B1B68DB6A9A42CDD9069BE4
:10BCF0004BB10123069A1360C7E700F118010A4807
:10BD0000074B9847EDE70122084B1A60BDE700BFDB
:10BD1000140E002009AA40001C0E0020A80D0020CF
:10BD2000BDA940009C0D0020540E0020840E002070
:10BD3000F8B5EFF311854FF0500383F31188BFF38B
:10BD40006F8FBFF34F8F90F85830DBB2022280F82C
:10BD50005820426D01324265012B02D085F31188D3
:10BD6000F8BD0E460446154B1B68E3B9071D38465F
:10BD7000134B9847E36A01229A401249086802432C
:10BD80000A6003EB83039A0039460F4810440F4BB7
:10BD90009847E26A0E4B1B68DB6A9A42DED946B1CD
:10BDA00001233360DAE700F118010A48074B98478E
:10BDB000EFE70122084B1A60D0E700BF140E002005
:10BDC00009AA40001C0E0020A80D0020BDA94000BB
:10BDD0009C0D0020540E0020840E0020064BDB6BCF
:10BDE000C3F30023054A1370054BDB6BC3F34033E9
:10BDF000044A1370704700BF00100E40880E0020E8
:10BE0000000E0E40890E002008B5054BDB6B13F4C5
:10BE1000004F02D1034B984708BD034B984708BD1C
:10BE2000000E0E404D4D4000714D400030B583B0C6
:10BE300004460D46002301932E4B984213D02E4BFF
:10BE40009C421AD02D4B9C4221D02D4B9C4228D095
:10BE50002C4B9C422FD02C4B9C4236D02B4B9C42DF
:10BE60003DD003B030BD01A92046294B984700289A
:10BE7000F9D19DF804302B70E1E701A92046244B4D
:10BE800098470028F9D19DF804302B70DAE701A912
:10BE900020461F4B98470028F9D19DF804302B709D
:10BEA000D3E701A920461A4B98470028F9D19DF8FD
:10BEB00004302B70CCE701A92046154B9847002889
:10BEC000F9D19DF804302B70C5E701A92046104B2D
:10BED00098470028F9D19DF804302B70BEE701A9DE
:10BEE00020460B4B98470028F9D19DF804302B7061
:10BEF000B7E700BF00C2004000020240004202401B
:10BF00000082014000C20140008200400002044063
:10BF100061A6400038B504460D46274B984213D021
:10BF2000264B984218D0264B98421DD0254B98425C
:10BF300022D0254B984227D0244B98422CD0244B1A
:10BF4000984231D0002038BD29462046214B9847E1
:10BF50000028F9D1012038BD294620461D4B9847BD
:10BF60000028F9D1012038BD29462046194B9847B1
:10BF70000028F9D1012038BD29462046154B9847A5
:10BF80000028F9D1012038BD29462046114B984799
:10BF90000028F9D1012038BD294620460D4B98478D
:10BFA0000028F9D1012038BD29462046094B984781
:10BFB0000028F9D1012038BD00C200400002024033
:10BFC000004202400082014000C201400082004065
:10BFD0000002044039A6400000B583B002A9002346
:10BFE00041F8043D084B1868084B9847019B3BB14A
:10BFF0004FF08052064B1A60BFF34F8FBFF36F8F25
:10C0000003B05DF804FB00BF8C0E002031BD400082
:10C0100004ED00E070B58AB01D4B0FCB0AAC04E90B
:10C020000F001C4D1C4B1D601C4A1D4B1A601D4A05
:10C030001D4B1A60069B0093079B0193089B02937C
:10C04000099B039300240494184E3046184B9847DC
:10C0500001213046174B9847174A69462846174B27
:10C0600098472846164B98472846164B9847164E31
:10C07000336821469868154DA847336821465868AB
:10C08000A847336821469868A8470AB070BD00BF2A
:10C090003804410000820140601B002015BF4000B1
:10C0A0005C1B00202DBE4000581B0020008001407A
:10C0B00021A2400089A340000000DC05C5A6400085
:10C0C00011A640001DA640000802002065DA4000CD
:10C0D00008B50A4601460248024B9847FEE700BFF2
:10C0E000DC0441003DD14000704770472DE9F0432A
:10C0F00083B0554B9847554A936843F0254343F422
:10C1000080139360524B9847524B98470120524BF3
:10C110009847524B98470446514B9847002800F0E7
:10C12000908094F89930002B40F0878094F89740E5
:10C130004C4B98474C4B98474C4B98474C4B984727
:10C1400005464C4B9847F022014628464A4B9847F3
:10C150004A4B98474A4B984720464A4B98474A488B
:10C160004A4B03602223037123234371484D294620
:10C17000484CA0474848494B03602B2303712A23AE
:10C1800043712946A047464B9847464B9847464837
:10C19000464B98474648474CA04747494748A04721
:10C1A000474A48494848A047002301930422009287
:10C1B0004FF4807245494648464CA047012802D0BA
:10C1C00045483C4B98474148444B9847444B18607E
:10C1D000444B9847444B9847444A00210F20444E13
:10C1E000B047444C03220B212046434DA847DFF8BB
:10C1F00018914A4600212820B047404F03220C21C5
:10C200003846A8472820DFF80481C0470146384651
:10C210003B4FB8474A4600210D20B04703220B216F
:10C220002046A8470D20C04701462046B847354B59
:10C230009847002003B0BDE8F0830020064B9847E4
:10C2400074E7502474E700BF9146400010140E407C
:10C25000A1A04000E56A4000414D4000C15D4000A2
:10C26000955E40004D4D400015C04000E97740000C
:10C270005179400059794000617840007D78400054
:10C28000E54B4000954C4000781B00200000024028
:10C29000A086010069674000641B002000C00140C7
:10C2A000ED7F400071444000D9BF4000854640000A
:10C2B000480441003DD1400064044100780441003D
:10C2C000800441008C04410098044100B004410006
:10C2D000657940005DB44000B804410055B74000A6
:10C2E0008C0E00207D724000E562400009BE4000D7
:10C2F0003D834000000E0E40AD83400000100E4014
:10C300001FA04000D1B44000DDBD400043A040006C
:10C3100000487047781B002000487047641B0020CD
:10C3200008B5014B984708BD6179400008B5014B3D
:10C33000984708BD637940000120704708B502485E
:10C34000024B984708BD00BF781B00205D68400085
:10C3500008B50248024B984708BD00BF641B002087
:10C360005D684000014B1878704700BF890E0020BF
:10C37000014B1878704700BF880E002070B58AB056
:10C38000044600F06FF8324B93F900506B1C0646E0
:10C3900009D02146204600F08DFE20B9002120461C
:10C3A00000F07EFE10B130460AB070BD294B0890F7
:10C3B0002046019300F006FBCDE90401CDE902011E
:10C3C0002046CDB9244B4FF060420021CDE9062331
:10C3D00000F03EFE002833D002230093684600F0B0
:10C3E00085F9A8B1089BC3B9DDE9060100F03EFB61
:10C3F000064630460AB070BD184B00220021CDE938
:10C40000062300F025FE68B102239D420093E5D18A
:10C4100000F066FE22230360E4E700F061FE089B63
:10C420000360E1E70123022D00930BD100F058FED9
:10C43000212303600A4800F05BF9CDE90601D1E74A
:10C4400001230093684600F051F90028F2D1EDE78E
:10C4500004020020F4044100FFFFEFC70000F0FFDA
:10C46000600441002DE9F84F30F000432DD0002842
:10C47000014604464ADBB0F1FF4F3BDAB0F5000F4E
:10C480003CDB00268D4AC4F316052A4402F4000260
:10C49000E41582F07E507F3C34444FF07E512843B7
:10C4A00004EBD25400F036FB05F10F03C3F316037F
:10C4B0000F2B064631DC002100F0CAFD002800F0F9
:10C4C00094804CB90020BDE8F88F00214FF04C401B
:10C4D00000F0DEFCBDE8F88F204600F0D1FB784983
:10C4E000054600F021FC77490446284600F01CFC74
:10C4F0000146204600F010FBBDE8F88F4FF0984150
:10C5000000F012FC6FF018060446BBE700F002FBD7
:10C51000002100F0BDFCBDE8F88F4FF0804100F035
:10C52000FBFA0146304600F0B3FC8046204600F09E
:10C53000A7FB41468146404600F0F6FB0146834694
:10C5400000F0F2FB6049DFF8A0A1074600F0ECFB29
:10C550005E4900F0E1FA394600F0E6FB5C4900F084
:10C56000DBFA394600F0E0FB5A4900F0D5FA5946AB
:10C5700000F0DAFB58498346384600F0D5FB5749AE
:10C5800000F0CAFA394600F0CFFB554900F0C4FA72
:10C59000394600F0C9FB0146584600F0BDFAC5F522
:10C5A0005713AA4403F5227343EA0A03002B0746F4
:10C5B00065DD4FF07C51304600F0B6FB314600F0AF
:10C5C000B3FB0546002C32D12946384600F0A4FAC8
:10C5D000414600F0A9FB0146284600F09BFA0146BF
:10C5E000304600F097FABDE8F88F3E49304600F03B
:10C5F0009BFB01464FF07C5000F08CFA314605461B
:10C60000304600F091FB0146284600F08DFB0546C0
:10C61000002C2ED0204600F033FB2949074600F0BD
:10C6200083FB28490446384600F07EFB14E0244989
:10C63000484600F079FB29460446384600F06CFA7B
:10C64000414600F071FB1F490746484600F06CFB6D
:10C650000146384600F060FA0146284600F05AFAD2
:10C66000314600F057FA0146204600F053FABDE883
:10C67000F88F0146304600F04DFABDE8F88F7CB1E6
:10C680000F49484600F050FB39460446304600F05A
:10C6900041FA414600F048FB0A4905464846C3E7CF
:10C6A0000146304600F036FA414600F03DFB0146B7
:10C6B000304600F02FFABDE8F88F00BF20FB4A009B
:10C6C0008071313FD1F717379788173E25333A3EAF
:10C6D0002549923EABAA2A3F4FD01C3E298E633E8D
:10C6E000CDCCCC3EABAAAA3E305CCFFF0020704739
:10C6F00000200149704700BF0000F87F81F0004131
:10C7000002E000BF83F0004330B54FEA41044FEA36
:10C71000430594EA050F08BF90EA020F1FBF54EAD1
:10C72000000C55EA020C7FEA645C7FEA655C00F06D
:10C73000E2804FEA5454D4EB5555B8BF6D420CDD3E
:10C740002C4480EA020281EA030382EA000083EAC1
:10C75000010180EA020281EA0303362D88BF30BD61
:10C7600011F0004F4FEA01314FF4801C4CEA1131B7
:10C7700002D0404261EB410113F0004F4FEA033316
:10C780004CEA133302D0524263EB430394EA050FA1
:10C7900000F0A780A4F10104D5F1200E0DDB02FA10
:10C7A0000EFC22FA05F2801841F1000103FA0EF2A4
:10C7B000801843FA05F359410EE0A5F120050EF16A
:10C7C000200E012A03FA0EFC28BF4CF0020C43FA9B
:10C7D00005F3C01851EBE37101F0004507D54FF0A8
:10C7E000000EDCF1000C7EEB00006EEB0101B1F5F8
:10C7F000801F1BD3B1F5001F0CD349085FEA30003E
:10C800004FEA3C0C04F101044FEA445212F5800F48
:10C8100080F09A80BCF1004F08BF5FEA500C50F1E5
:10C82000000041EB045141EA050130BD5FEA4C0CC8
:10C83000404141EB010111F4801FA4F10104E9D151
:10C8400091F0000F04BF01460020B1FA81F308BF48
:10C850002033A3F10B03B3F120020CDA0C3208DD14
:10C8600002F1140CC2F10C0201FA0CF021FA02F1EF
:10C870000CE002F11402D8BFC2F1200C01FA02F15F
:10C8800020FA0CFCDCBF41EA0C019040E41AA2BF84
:10C8900001EB0451294330BD6FEA04041F3C1CDA4C
:10C8A0000C340EDC04F11404C4F1200220FA04F06C
:10C8B00001FA02F340EA030021FA04F345EA030116
:10C8C00030BDC4F10C04C4F1200220FA02F001FAD8
:10C8D00004F340EA0300294630BD21FA04F029465A
:10C8E00030BD94F0000F83F4801306BF81F48011F3
:10C8F0000134013D4EE77FEA645C18BF7FEA655C66
:10C9000029D094EA050F08BF90EA020F05D054EA37
:10C91000000C04BF1946104630BD91EA030F1EBF3C
:10C920000021002030BD5FEA545C05D14000494140
:10C9300028BF41F0004130BD14F580043CBF01F533
:10C94000801130BD01F0004545F0FE4141F4700119
:10C950004FF0000030BD7FEA645C1ABF19461046F4
:10C960007FEA655C1CBF0B46024650EA013406BFF5
:10C9700052EA033591EA030F41F4002130BD00BFB4
:10C9800090F0000F04BF0021704730B54FF4806471
:10C9900004F132044FF000054FF0000150E700BFF2
:10C9A00090F0000F04BF0021704730B54FF4806451
:10C9B00004F1320410F0004548BF40424FF000013E
:10C9C0003EE700BF42004FEAE2014FEA31014FEA81
:10C9D00002701FBF12F07F4393F07F4F81F06051D0
:10C9E000704792F0000F14BF93F07F4F704730B53F
:10C9F0004FF4607401F0004521F0004120E700BFD2
:10CA000050EA010208BF704730B54FF000050AE058
:10CA100050EA010208BF704730B511F0004502D559
:10CA2000404261EB41014FF4806404F132045FEA5B
:10CA3000915C3FF4DCAE4FF003025FEADC0C18BF00
:10CA400003325FEADC0C18BF033202EBDC02C2F1F6
:10CA5000200300FA03FC20FA02F001FA03FE40EA88
:10CA60000E0021FA02F11444C1E600BF4FEA410270
:10CA7000B2F1E04324BFB3F5001CDCF1FE5C0DD93C
:10CA800001F0004C4FEAC0024CEA5070B2F1004F86
:10CA900040EB830008BF20F00100704711F0804F89
:10CAA00021D113F13872BCBF01F00040704741F44E
:10CAB00080114FEA5252C2F11802C2F1200C10FA52
:10CAC0000CF320FA02F018BF40F001004FEAC12336
:10CAD0004FEAD32303FA0CFC40EA0C0023FA02F3DA
:10CAE0004FEA4303CCE77FEA625307D150EA0133B0
:10CAF0001EBF4FF0FE4040F44000704701F0004080
:10CB000040F0FE4040F40000704700BF80F000405D
:10CB100002E000BF81F0004142001FBF5FEA410315
:10CB200092EA030F7FEA226C7FEA236C6AD04FEA15
:10CB30001262D2EB1363C1BFD2184140484041405A
:10CB4000B8BF5B42192B88BF704710F0004F40F40C
:10CB5000000020F07F4018BF404211F0004F41F428
:10CB6000000121F07F4118BF494292EA030F3FD0F4
:10CB7000A2F1010241FA03FC10EB0C00C3F1200307
:10CB800001FA03F100F0004302D5494260EB400096
:10CB9000B0F5000F13D3B0F1807F06D340084FEA01
:10CBA000310102F10102FE2A51D2B1F1004F40EBF6
:10CBB000C25008BF20F0010040EA0300704749005E
:10CBC00040EB000010F4000FA2F10102EDD1B0FA29
:10CBD00080FCACF1080CB2EB0C0200FA0CF0AABF1E
:10CBE00000EBC25052421843BCBFD04018437047BC
:10CBF00092F0000F81F4000106BF80F400000132C2
:10CC0000013BB5E74FEA41037FEA226C18BF7FEA98
:10CC1000236C21D092EA030F04D092F0000F08BFDA
:10CC20000846704790EA010F1CBF0020704712F0C1
:10CC30007F4F04D1400028BF40F00040704712F100
:10CC400000723CBF00F50000704700F0004343F065
:10CC5000FE4040F4000070477FEA226216BF08469B
:10CC60007FEA23630146420206BF5FEA412390EA5E
:10CC7000010F40F4800070474FF0000304E000BF54
:10CC800010F0004348BF40425FEA000C08BF704705
:10CC900043F0964301464FF000001CE050EA0102C9
:10CCA00008BF70474FF000030AE000BF50EA0102DE
:10CCB00008BF704711F0004302D5404261EB4101CB
:10CCC0005FEA010C02BF84460146002043F0B643F0
:10CCD00008BFA3F18053A3F50003BCFA8CF2083A15
:10CCE000A3EBC25310DB01FA02FC634400FA02FC1E
:10CCF000C2F12002BCF1004F20FA02F243EB020025
:10CD000008BF20F00100704702F1200201FA02FC86
:10CD1000C2F1200250EA4C0021FA02F243EB020079
:10CD200008BF20EADC7070474FF0FF0C1CEAD052BD
:10CD30001EBF1CEAD15392EA0C0F93EA0C0F6FD07E
:10CD40001A4480EA010C400218BF5FEA41211ED05C
:10CD50004FF0006343EA501043EA5111A0FB013148
:10CD60000CF00040B1F5000F3EBF490041EAD3711D
:10CD70005B0040EA010062F17F02FD2A1DD8B3F199
:10CD8000004F40EBC25008BF20F00100704790F008
:10CD9000000F0CF0004C08BF49024CEA502040EA5A
:10CDA00051207F3AC2BFD2F1FF0340EAC250704720
:10CDB00040F400004FF00003013A5DDC12F1190F5E
:10CDC000DCBF00F000407047C2F10002410021FAD0
:10CDD00002F1C2F1200200FA02FC5FEA310040F1E8
:10CDE000000053EA4C0308BF20EADC70704792F061
:10CDF000000F00F0004C02BF400010F4000F013A99
:10CE0000F9D040EA0C0093F0000F01F0004C02BF93
:10CE1000490011F4000F013BF9D041EA0C018FE702
:10CE20000CEAD15392EA0C0F18BF93EA0C0F0AD008
:10CE300030F0004C18BF31F0004CD8D180EA01002E
:10CE400000F00040704790F0000F17BF90F0004FC7
:10CE5000084691F0000F91F0004F14D092EA0C0FA9
:10CE600001D142020FD193EA0C0F03D14B0218BF3C
:10CE7000084608D180EA010000F0004040F0FE4082
:10CE800040F40000704740F0FE4040F4400070471E
:10CE90004FF0FF0C1CEAD0521EBF1CEAD15392EA9D
:10CEA0000C0F93EA0C0F69D0A2EB030280EA010C8D
:10CEB00049024FEA402037D04FF0805343EA111126
:10CEC00043EA10130CF000408B4238BF5B0042F184
:10CED0007D024FF4000C8B4224BF5B1A40EA0C0029
:10CEE000B3EB510F24BFA3EB510340EA5C00B3EB5B
:10CEF000910F24BFA3EB910340EA9C00B3EBD10F49
:10CF000024BFA3EBD10340EADC001B0118BF5FEA9A
:10CF10001C1CE0D1FD2A3FF650AF8B4240EBC250C3
:10CF200008BF20F0010070470CF0004C4CEA502084
:10CF30007F32C2BFD2F1FF0340EAC250704740F4D3
:10CF400000004FF00003013A37E792F0000F00F0C5
:10CF5000004C02BF400010F4000F013AF9D040EA43
:10CF60000C0093F0000F01F0004C02BF490011F4D7
:10CF7000000F013BF9D041EA0C0195E70CEAD153CF
:10CF800092EA0C0F08D142027FF47DAF93EA0C0FB6
:10CF90007FF470AF084676E793EA0C0F04D14B029A
:10CFA0003FF44CAF08466EE730F0004C18BF31F04C
:10CFB000004CCAD130F000427FF45CAF31F0004346
:10CFC0007FF43CAF5FE700BF4FF0FF3C06E000BFDF
:10CFD0004FF0010C02E000BF4FF0010C4DF804CD02
:10CFE0004FEA40024FEA41037FEA226C18BF7FEA12
:10CFF000236C11D001B052EA530C18BF90EA010F14
:10D0000058BFB2EB030088BFC81738BF6FEAE170A2
:10D0100018BF40F0010070477FEA226C02D15FEA3E
:10D02000402C05D17FEA236CE4D15FEA412CE1D0AA
:10D030005DF8040B704700BF844608466146FFE771
:10D040000FB5FFF7C9FF002848BF10F1000F0FBD53
:10D050004DF808EDFFF7F4FF0CBF012000205DF84C
:10D0600008FB00BF4DF808EDFFF7EAFF34BF0120D1
:10D0700000205DF808FB00BF4DF808EDFFF7E0FF6A
:10D0800094BF012000205DF808FB00BF4DF808EDBB
:10D09000FFF7D2FF94BF012000205DF808FB00BF1E
:10D0A0004DF808EDFFF7C8FF34BF012000205DF800
:10D0B00008FB00BF4FEA40024FEA41037FEA226CBF
:10D0C00002D15FEA402C08D17FEA236C02D15FEAEB
:10D0D000412C02D14FF0000070474FF00100704723
:10D0E000014B1868704700BF0802002070B50F4E52
:10D0F0000F4D761BB61018BF002405D0013455F82B
:10D10000043B9847A642F9D10A4E0B4D761B03F01B
:10D11000A9FAB61018BF002406D0013455F8043B14
:10D120009847A642F9D170BD70BD00BF700641009E
:10D130007006410078064100700641000FB400B54A
:10D14000074983B004AB086853F8042B8168019346
:10D1500000F024FE03B05DF804EB04B0704700BF9C
:10D1600008020020024B0146186800F00BB800BF0F
:10D1700008020020024B0146186801F02BBF00BFD7
:10D18000080200202DE9F04F01F10B06162E83B0A6
:10D19000054640F29E8036F0070600F1BD80B142A0
:10D1A00000F2BA8000F040FCB6F5FC7FC0F093823C
:10D1B000730A00F0B880042B00F27981B30903F1FF
:10D1C000390003F1380EC300BF4F3B44A3F10801FF
:10D1D0005C68A14206D10CE0002A80F2AA80E468D3
:10D1E000A14206D0636823F003039A1B0F2AF3DDE4
:10D1F00070463C69DFF8E4E2744500F0AB81636897
:10D2000023F003039A1B0F2A00F39081002AC7F82A
:10D2100014E0C7F810E080F29D80B3F5007F80F045
:10D220006181DB0803F1010C99107A6857F83C80A2
:10D23000C4F8088001238B4007EBCC011343083965
:10D24000E1607B6047F83C40C8F80C408210012444
:10D2500094409C4200F28B801C4206D120F00300D7
:10D2600064001C4200F10400FAD007EBC009CC4670
:10D270008046DCF80C309C4507D16DE1002A80F235
:10D280007B81DB689C4500F06781596821F00301D0
:10D290008A1B0F2AF2DDD3F80CC0D3F80880009364
:10D2A0009C19284646F0010642F001055E60C8F868
:10D2B0000CC0CCF808807C613C61C4F80CE0C4F878
:10D2C00008E065605A5000F0B5FB009B03F10804CC
:10D2D0001EE0102920D800F0A7FB102618230220FA
:10D2E000794F3B44A3F108025C68944200F03D8111
:10D2F0006368E168A66823F00303234428465A685C
:10D30000F16042F001028E605A6000F093FB083435
:10D31000204603B0BDE8F08F00240C2320462B608C
:10D3200003B0BDE8F08F40204FF400734FF03F0E84
:10D330004AE72344E1685A68A66842F00102F160B6
:10D3400028468E605A6000F075FB0834204603B012
:10D35000BDE8F08F234428465A6842F001025A6023
:10D3600000F068FB0834204603B0BDE8F08FBC68CD
:10D37000636823F00308B04504D3A8EB06030F2B22
:10D3800000F38580DFF85891504BD9F800201B68D6
:10D390000132334404EB080A00F0558103F5805351
:10D3A0000F3323F47F6B2BF00F0B5946284600F008
:10D3B00047FB411C024600F0FC80824500F2F780EA
:10D3C000434B19685944196000F04D81D9F80000A9
:10D3D00001301BBFA2EB0A0A5144C9F800201960B2
:10D3E00012F0070100F01581C1F10800C1F580516C
:10D3F0000244083102EB0B09C9F30B09A1EB09093F
:10D40000494628460193009200F01AFB431C9DE810
:10D410000C0000F04381801A484440F00100196874
:10D42000BA604944BC425060196017D0B8F10F0F80
:10D4300040F2FB806068A8F10C0222F0070204EBC6
:10D44000020E00F001004FF0050C10430F2A60603F
:10D45000CEF804C0CEF808C000F217811D4BBC689E
:10D460001A68914288BF19601B4B1A689142626822
:10D4700088BF196022F003029642A2EB060301D88E
:10D480000F2B04DC284600F0D5FA002440E7A2194F
:10D4900043F0010346F0010666602846BA60536017
:10D4A00000F0C8FA0834204603B0BDE8F08F142B12
:10D4B00071D9542B00F2A380330B03F16F0003F1F9
:10D4C0006E0EC30080E600BF38060020C00E0020AC
:10D4D000900E0020B80E0020BC0E00204006002058
:10D4E000400A00205A0A042A5BD9142A00F2AE80AE
:10D4F00002F15C01C9005B3207EB010C7958ACF119
:10D50000080C8C4500F088804A6822F003029342A0
:10D5100073D289688C45F7D1DCF80C207B68E26017
:10D52000C4F808C09460CCF80C408FE6A11946F00E
:10D53000010C42F00106C4F804C028467961396143
:10D54000C1F80CE0C1F808E04E60E25000F072FA59
:10D550000834DDE67B6879E608F1010818F0030F6E
:10D560000CF1080C7FF485AE2DE0DC68A34208BF07
:10D5700002303FF43EAEBBE619441C464A68DB6805
:10D5800054F8086F42F001024A602846F3609E603A
:10D5900000F050FABCE603F15C0003F15B0EC3003F
:10D5A00012E69A0902F13901C9003832A4E7BC42F7
:10D5B00054D0BC68626822F003025DE759F808396C
:10D5C000994540F0868010F0030F00F1FF30F5D14F
:10D5D0007B6823EA04037B6064009C423FF6C7AE8D
:10D5E000002C3FF4C4AE1C4240467FF43EAE6400C3
:10D5F0001C4200F10400FAD037E68C468CE7B3F504
:10D60000AA7F15D8F30B03F1780003F1770EC3005E
:10D61000DAE54FF48051EDE67B689210012101FAC2
:10D6200002F213437B60624679E70123536029E7E6
:10D6300040F25452934222D8B30C03F17D0003F11F
:10D640007C0EC300C0E503F1100BAEE6542A29D8C6
:10D650001A0B02F16F01C9006E324DE7204B1968B9
:10D6600059441960B2E6CAF30B0000287FF4AEAE4D
:10D6700008EB0B03BA6843F001035360EEE67F202A
:10D680004FF47E734FF07E0E9EE504F108012846AC
:10D69000009301F09FFC009B1968DFE601204FF02A
:10D6A0000009BCE6B2F5AA7F05D8DA0B02F17801D1
:10D6B000C900773220E740F254518A4205D89A0CCB
:10D6C00002F17D01C9007C3216E74FF47E717E22A3
:10D6D00012E77B6880E7F00806F1080300E600BF68
:10D6E000900E00200000000000000000000000007C
:10D6F00001F0FF01102A2BDB10F0070F08D010F803
:10D70000013B013A8B422DD010F0070F42B3F6D106
:10D71000F0B441EA012141EA014122F007047FF01F
:10D7200000070023F0E80256083C85EA010586EA76
:10D73000010685FA47F5A3FA87F586FA47F6A5FAB2
:10D7400087F68EB9EED1F0BC01F0FF0102F00702BE
:10D7500032B110F8013B013A83EA010313B1F8D169
:10D760000020704701387047002D06BF354603384A
:10D77000073815F0010F07D1013015F4807F02BF83
:10D78000013015F4C03F0130F0BC0138704700BFD4
:10D79000844641EA000313F003036DD1403A41D3BC
:10D7A00051F8043B40F8043B51F8043B40F8043B7B
:10D7B00051F8043B40F8043B51F8043B40F8043B6B
:10D7C00051F8043B40F8043B51F8043B40F8043B5B
:10D7D00051F8043B40F8043B51F8043B40F8043B4B
:10D7E00051F8043B40F8043B51F8043B40F8043B3B
:10D7F00051F8043B40F8043B51F8043B40F8043B2B
:10D8000051F8043B40F8043B51F8043B40F8043B1A
:10D8100051F8043B40F8043B51F8043B40F8043B0A
:10D82000403ABDD2303211D351F8043B40F8043BAA
:10D8300051F8043B40F8043B51F8043B40F8043BEA
:10D8400051F8043B40F8043B103AEDD20C3205D3BA
:10D8500051F8043B40F8043B043AF9D2043208D0B2
:10D86000D2071CBF11F8013B00F8013B01D30B8824
:10D8700003806046704700BF082A13D38B078DD002
:10D8800010F003038AD0C3F10403D21ADB071CBFD4
:10D8900011F8013B00F8013B80D331F8023B20F83E
:10D8A000023B7BE7043AD9D3013A11F8013B00F877
:10D8B000013BF9D20B7803704B7843708B788370FF
:10D8C000604670478842F0B50DD98B1898420AD24D
:10D8D0008418002A51D0224613F8014D02F8014D58
:10D8E0009942F9D1F0BD0F2A48D941EA00039B07BC
:10D8F00046D100F1100401F11003154653F8106CE5
:10D9000044F8106C53F80C6C44F80C6C53F8086C29
:10D9100044F8086C103D53F8046C44F8046C0F2D67
:10D9200003F1100304F11004E8D8A2F1100323F06E
:10D930000F0302F00F0E1033BEF1030F194403441E
:10D9400021D91E1F0D467446043C55F8047B46F849
:10D95000047F032CF8D8AEF1040424F0030404344B
:10D960002144234402F0030262B1013B0A4411F84E
:10D97000014B03F8014F8A42F9D1F0BD0346F3E7AA
:10D980000346F2E7F0BD7246EEE700BF70B48607CB
:10D9900046D0541E002A41D0CAB2034602E014F118
:10D9A000FF343BD303F8012B9D07F8D1032C2ED96C
:10D9B000CDB245EA05250F2C45EA054519D903F1F5
:10D9C00010022646103E0F2E42F8105C42F80C5C06
:10D9D00042F8085C42F8045C02F11002F2D8A4F1AB
:10D9E000100222F00F0204F00F041032032C134433
:10D9F0000DD91E462246043A032A46F8045BFAD89B
:10DA0000221F22F003020432134404F003042CB159
:10DA1000C9B21C4403F8011B9C42FBD170BC704787
:10DA200014460346C2E700BF014801F06DBD00BFC8
:10DA30009C1B0020014801F069BD00BF9C1B002019
:10DA400038B5074C0023054608462360FCF780FFE5
:10DA5000431C00D038BD2368002BFBD02B6038BDA1
:10DA6000B01B002000290CBF022200224FF480636B
:10DA700000F000B82DE9F043614C256883B00446FE
:10DA80000F4690461E4615B1AB6B002B64D0B8F123
:10DA9000020F06D0B8F1010F00F29F80002EC0F2F5
:10DAA0009C80636ED80734D52146284601F014F9CE
:10DAB000216B41B104F14003994202D0284601F0A4
:10DAC00089FA00232363B4F90C300022A26162605A
:10DAD0001A063AD423F44A6323F00303B8F1020F81
:10DAE000A3811DD001AB6A462146284601F010FDF6
:10DAF000A3891843A081002E32D1009E3046FFF743
:10DB000031FB074600286BD0A38943F08003A38133
:10DB100028E0A3899905C7D4A06D01F0F5FCC3E7FF
:10DB20000025616E002604F1430243F00203012048
:10DB3000A660CE07A38122602261606101D49805AE
:10DB40003ED5284603B0BDE8F0832169284601F0A0
:10DB500041FAB4F90C30BDE7284601F015F996E713
:10DB6000002FCBD0AB6B002B33D0009BB4F90C2033
:10DB700027609E421CBF42F40062A281B8F1010FEF
:10DB800004BF42F00102A28192B212F008032761A1
:10DB900066610ED0D1071AD5656E7642002315F066
:10DBA0000105A661A36009D00025284603B0BDE8A1
:10DBB000F083A360656E15F00105F5D19305C0D41F
:10DBC000A06D01F0A3FC284603B0BDE8F083A66079
:10DBD000F0E7284601F0D8F8C7E74FF0FF35B0E787
:10DBE000DDF80090B14504D04846FFF7BBFA074680
:10DBF00020B9B4F90C304FF0FF3592E74E4683E779
:10DC000008020020000000000000000000000000EA
:10DC10000000000000000000000000000000000004
:10DC200000000000000000000000000000000000F4
:10DC300000000000000000000000000000000000E4
:10DC400090F800F06DE9024520F007016FF0000C3C
:10DC500010F0070491F820F040F049804FF00004E4
:10DC60006FF00700D1E9002391F840F000F10800BF
:10DC700082FA4CF2A4FA8CF283FA4CF3A2FA8CF3F7
:10DC80004BBBD1E9022382FA4CF200F10800A4FA5E
:10DC90008CF283FA4CF3A2FA8CF3E3B9D1E90423B2
:10DCA00082FA4CF200F10800A4FA8CF283FA4CF3E9
:10DCB000A2FA8CF37BB9D1E9062301F1200182FAA3
:10DCC0004CF200F10800A4FA8CF283FA4CF3A2FAA9
:10DCD0008CF3002BC6D0002A04BF04301A4612BAB7
:10DCE000B2FA82F2FDE8024500EBD2007047D1E9BA
:10DCF000002304F00305C4F100004FEAC50514F049
:10DD0000040F91F840F00CFA05F562EA05021CBF19
:10DD100063EA050362464FF00004A9E72DE9F84FD6
:10DD20004B6E9C0493462FD59368126853B30E46EE
:10DD3000074602F1080919E920045FEA9A0817D09A
:10DD4000043D002401E0A04510D0324655F8041FE0
:10DD5000384601F0BBF8431C04F10104F3D1002361
:10DD6000CBF80830CBF80430BDE8F88FDBF808308A
:10DD70002AF0030AA3EB0A03CBF8083009F10809DB
:10DD8000002BD8D10020EAE701F00AFA0023CBF8F3
:10DD90000830CBF80430BDE8F88F00BF2DE9F04F14
:10DDA000ADB01D468B4690460793069018B1836B25
:10DDB000002B00F0F380DBF86430BBF90C00DF07C8
:10DDC00081B202D48E0540F1FC808C040AD4DBF8C9
:10DDD000643040F4005123F40053ABF80C10CBF83E
:10DDE000643089B2080740F1B380DBF81030002BB3
:10DDF00000F0AE8001F01A030A2B00F0B58000237A
:10DE00000DF170090B93119310930393CDF83C908F
:10DE1000CA46CDF810B098F800304446FBB1252B27
:10DE200002D11CE0252B03D014F8013F002BF9D1BF
:10DE3000A4EB08059DB1109B119ACAF8008001332C
:10DE40002A44072BCAF80450119210937ADD002A55
:10DE500040F0B084039B10922B44CA46039323786E
:10DE6000002B00F0E08300204FF000038DF83730E6
:10DE700004F1010862780546064603464FF0FF3478
:10DE800008F10108A2F12001582900F2DE82DFE842
:10DE900011F02102DC02DC022902DC02DC02DC02DD
:10DEA000DC02DC02DC0289029502DC02A200BD0277
:10DEB000DC029F01A401A401A401A401A401A40106
:10DEC000A401A401A401DC02DC02DC02DC02DC020D
:10DED000DC02DC02DC02DC02DC02B201DC02DC027D
:10DEE000DC02DC02DC02DC02DC02DC02DC02DC0242
:10DEF0009701DC02DC02DC02DC02DC029B01DC02BA
:10DF0000DC025302DC02DC02DC02DC02DC02DC02AA
:10DF1000DC02DC02DC02DC025A021B02DC02DC0254
:10DF2000DC026E021B02DC02DC027302DC02F50181
:10DF300082010902D702DC029A02DC02A700DC029D
:10DF4000DC022E020AF1080A039B2B44039386E7A6
:10DF50005946069800F0ACFD18BBBBF80C1001F058
:10DF60001A030A2B7FF44BAFBBF90E30002BFFF6E0
:10DF700046AFDBF86430DB0705D48F0503D4DBF84C
:10DF8000580001F0C3FA2B4642465946069800F065
:10DF90004DFD039003982DB0BDE8F08F00F0F4FE26
:10DFA00009E7DBF86430D90704D4BBF80C309A05D4
:10DFB00040F1AA844FF0FF33039303982DB0BDE8DE
:10DFC000F08FDBF8580001F09FFABBF90C0081B22A
:10DFD000FBE67642079243F0040398F800204FE7EF
:10DFE00008969E0600F150840799DD060A4600F166
:10DFF000EF83580640F1EC830E880431002701229C
:10E0000007914FF000018DF837100025611C00F0DA
:10E01000168123F08001029156EA070140F0148135
:10E02000002C40F05C83002A40F0B78313F001031A
:10E03000059300F057840DF1B00B30230BF8413DF0
:10E04000059BA342B8BF234601930DB10133019351
:10E05000029B13F00203099302D0019B0233019348
:10E06000029B13F084030A9340F01782089B019AE5
:10E070009D1A002D40F31182102D40F39084109BC7
:10E08000119AC44ED6461027A2461946069C07E0B0
:10E0900001F1020C0EF1080E0146103D102D11DDAC
:10E0A000481C1032072811928EE8C0001090EFDD56
:10E0B000002A40F0E481103D102D11464FF0010C74
:10E0C000CE46EDDC54466146F2462A4407291192B9
:10E0D000CAF80060CAF80450109100F3EC829DF871
:10E0E00037500AF1080A481C002D40F0DE81099BD8
:10E0F000002B00F0F88102320EA9022307281192AA
:10E1000010908AE80A0040F3EA81002A40F08C83EC
:10E110000A9B802B4FF001001146CA4640F0E78170
:10E12000089B019D5E1B002E40F3E181102E9A4D4D
:10E1300040F35084D4461027A246069C07E001F124
:10E14000020E0CF1080C0146103E102E11DD481C89
:10E150001032072811928CE8A0001090EFDD002A01
:10E1600040F09D82103E102E4FF0010E1146CC461D
:10E17000EDDC5446E2463244BEF1070F11928AE8C4
:10E180006000CDF840E000F369830AF1080A0EF15F
:10E1900001007146ABE1089613F0200240F08C8339
:10E1A00013F0100140F01A8313F0400200F01683C0
:10E1B00007980A460146043106880791002720E7A0
:10E1C000089643F01003E7E7089643F0100308E7CA
:10E1D00043F0800398F8002052E6A2F130010026B7
:10E1E00018F8012B06EB860601EB4606A2F130017A
:10E1F0000929F5D946E60896002840F0088443F03E
:10E2000010039E0600F14C83DD0600F1F3825806F0
:10E2100040F1F082079DB5F900602A46F7170432F5
:10E22000304639460792002871F10002C0F25D8342
:10E23000611C9DF837504FF001027FF4EAAE56EAB8
:10E24000070100F04D820293012A00F08C82022A1D
:10E2500040F05C820B98CB46330906F00F0143EA8D
:10E2600007733A091E461746435C0BF8013D56EA10
:10E270000703F1D1A9EB0B030593E1E6002840F079
:10E28000C083990600F16783DA0600F1F1805B062E
:10E2900040F1EE80079A136804320792BDF80C2013
:10E2A0001A80B8E507983D4A08960B9206687822CE
:10E2B000302104308DF8392043F002030790002705
:10E2C0008DF8381002229CE60896002899D08DF827
:10E2D000375096E798F80020002D7FF4D1AD01204B
:10E2E0002025CDE543F0010398F80020C8E5089605
:10E2F000002840F0938329490B919F0600F1E882A2
:10E300000798DE06014600F170825D0640F16D82DD
:10E310000431068807910027D80740F1228256EA87
:10E32000070100F01E8230218DF8392043F00203EE
:10E330008DF83810022264E60896002840F06B83BE
:10E3400017490B91D9E7079908960A688DF8482074
:10E350004FF000000A468DF837000432012001908A
:10E36000079205900DF1480B0293002470E643F0EC
:10E37000400398F8002083E598F800206C2A03BF3A
:10E3800098F8012043F0200308F1010843F010033E
:10E3900076E500BF3005410040054100140541000D
:10E3A0000005410007990E680A46002E02F104029A
:10E3B000FFF60FAE079298F8002061E598F800206C
:10E3C00001202B255CE507990896D1F800B04FF0A5
:10E3D00000028DF837200E1DBBF1000F00F0E58222
:10E3E000671C00F0C4822246002158460193FFF7C3
:10E3F0007FF9019B002800F0E582A0EB0B0205925B
:10E40000079602939DF83750002419E698F80020EB
:10E410002A2A08F1010700F0E982A2F13001092956
:10E42000B8464FF000043FF62DAD18F8012B04EB71
:10E43000840401EB4404A2F130010929F5D921E556
:10E4400043F0200398F800201AE50896002840F0D1
:10E45000DB82002A00F0E78001218DF848204FF090
:10E46000000201918DF8372005910DF1480B7BE7F3
:10E47000079A136804320792039A1A60CBE40FAA32
:10E4800004992046FFF74AFC002840F03981109992
:10E49000119A01F1010CCE46FFE51099119A481C22
:10E4A0009DF83750002D3FF422AE01320DF13705B3
:10E4B0000121072811921090CAF80050CAF80410E0
:10E4C00040F30881002A40F0BC81099B002B3FF4F7
:10E4D0001FAE0EAB022208461C931D92CA4601468F
:10E4E0000AF1080A01300A9B802B3FF419AE059B04
:10E4F000E41A002C2EDD102CB34D1EDDD64610265E
:10E50000069FDDF810A006E0881C0EF1080E1946E3
:10E51000103C102C10DD4B1C1032072B11928EE892
:10E5200060001093F0DD002A65D1103C102C4FF0F4
:10E5300001001146CE46EEDCF24622440728119235
:10E54000CAF80050CAF80440109000F385800AF120
:10E55000080A01300599CAF800B00A440728119248
:10E56000CAF80410109040F38280002A40F018810D
:10E57000029B1092580735D5089B01995C1A002C14
:10E5800040F3E780CA46102C40F3188210998F4E52
:10E59000069FDDF810B0102506E0881C0AF1080A75
:10E5A0001946103C102C11DD4B1C1032072B119218
:10E5B000CAF80060CAF804501093EEDD42BB103C6C
:10E5C000102C4FF001001146CA46EDDC224407280A
:10E5D0001192CAF80060CAF80440109051DD002A78
:10E5E00040F09B81039B089A01998A42ACBF9B181B
:10E5F0005B1803934EE00FAA51463846FFF78EFB97
:10E60000002840F03F811099119A481CCE467FE7C0
:10E610000FAA59463846FFF781FB60B91099119A45
:10E62000481CCA46BDE7119BDDF810B0002B40F036
:10E63000D48100231093DBF8643013F0010FBBF892
:10E640000C3002D19A0540F1DE805B063FF5B2AC9A
:10E6500003982DB0BDE8F08F002A40F00681059A9E
:10E660001D9201231192CDF870B01093CA460AF1A1
:10E67000080A029B590704D5089B01995C1A002CD3
:10E6800081DC039B089901988142ACBF5B181B1881
:10E69000039372BB00231093CA46FFF7BCBB0FAABB
:10E6A00004992046FFF73AFB50BB1099119A01F1EB
:10E6B000010ECC4648E5002A40F040819DF8371015
:10E6C000002900F01B8101220DF1370110461D9237
:10E6D0001C91CA4601460AF1080A013007E5029B6F
:10E6E000012A00F09880022A0DD10293002600270B
:10E6F000B0E50FAA04990698FFF710FB0028C9D0CF
:10E70000DDF810B097E7029300260027494600E0A5
:10E710005946F20842EA4772F80806F0070307462E
:10E720001646303356EA070201F8013C01F1FF3B7F
:10E73000EED1029AD6077FF59DAD302B3FF49AAD0E
:10E74000023930230BF8013CA9EB010305938B46FA
:10E7500076E4039B089A8A42ACBF9B185B1803932C
:10E7600098E702224DE4002F08BF0A2E52D3CB4671
:10E77000304639460A22002301F010FB30320BF8F4
:10E78000012D3046394600230A2201F007FB0646D8
:10E790000F4656EA0703EBD16CE50594CB464FE4F0
:10E7A0000FAA04990698FFF7B9FA0028A8D1119A80
:10E7B000CA465EE70FAA04990698FFF7AFFA002849
:10E7C0009ED1CA46FFF7C0BB40054100300541005D
:10E7D0000431166807910122002712E407980146C8
:10E7E00004310668079100270BE40E680431079195
:10E7F000002791E507990E680A46F7170432079239
:10E80000304639460FE5DBF8580000F07FFEBBF8D4
:10E810000C301AE7029B02930DF1B00B3036012346
:10E820000BF8416D05930BE40FAA04990698FFF7C6
:10E8300075FA00287FF464AF1099119A481CCA46F3
:10E8400051E60FAA04990698FFF768FA00287FF4AA
:10E8500057AF1099119A481CCA4648E4002A40F064
:10E86000918001201146CA4641E60FAA04990698F4
:10E87000FFF754FA00287FF443AF1098119A013043
:10E88000CA4667E6D346D6E6079E073626F0070255
:10E8900002F10801D2E9006707910122FFF7B1BB3D
:10E8A000079E073626F00706D6E9000106F10802A2
:10E8B000079206460F46B6E4079E073626F0070283
:10E8C00002F10801D2E9006707910022FFF799BB26
:10E8D000079E073626F0070101F108000790D1E9ED
:10E8E000006719E5CB46FFF7ABBB2D25764267EBFA
:10E8F00047078DF837500122FFF788BB099BB3B952
:10E9000011460120CA46F2E5DBF8580000F0FEFD92
:10E910004FF0FF330393FFF750BB0FAA04990698FB
:10E92000FFF7FCF900287FF4EBAE119AA9E60EABD5
:10E9300002221C931D920120CA46D0E50FAA049919
:10E940000698FFF7EBF900287FF4DAAE1099119AD8
:10E95000481CCA46A4E5079A03991368CD170846D0
:10E96000043229460792C3E90001FFF754BA58461A
:10E9700007960293FFF764F9002405909DF837503D
:10E98000FFF75EBB0FAA04990698FFF7C7F90028A6
:10E990007FF4B6AE1099119A481CCA46A7E51099A3
:10E9A000119A204E0131FFF790BB062C28BF062498
:10E9B000059407960194DFF870B0D5E41098194ECD
:10E9C000013003E605949DF83750079602930446FC
:10E9D000FFF736BB8646FFF7CEBB06980FAA59460F
:10E9E000FFF79CF900283FF424AE24E6079998F835
:10E9F00001200C68043144EAE474B8460791FFF73B
:10EA00003FBA8DF837503CE48DF8375021E58DF84A
:10EA10003750FFF7F4BB8DF8375091E48DF837503D
:10EA200069E400BF30054100280541002DE9F041AF
:10EA30000C46ADF58D6D8989666EE589199621F0D4
:10EA400002010646E069ADF80C1017464FF48061EC
:10EA5000626AADF80E5098461AAD0023079016A8CA
:10EA600009920693009504950291059100F048FDE6
:10EA700043463A4669463046FFF790F9051E07DBE4
:10EA80003046694600F028F9002818BF4FF0FF35DE
:10EA9000BDF80C305B0603D5A38943F04003A38186
:10EAA000169800F02FFD28460DF58D6DBDE8F0811C
:10EAB00038B5304B1B6805460C4613B19A6B002ADB
:10EAC00038D0B4F90C2093B218070CD52069A8B13E
:10EAD00013F001021ED0636900225B42A361A260B1
:10EAE000F0B1002038BDD9063CD5580726D420699E
:10EAF00042F00803A3819BB20028E9D103F42072FD
:10EB0000B2F5007FE4D02846214600F02FFDA3890E
:10EB10002069DDE7990758BF6269A2600028E0D14B
:10EB2000B4F90C301A06DDD543F04003A3814FF051
:10EB3000FF3038BD184600F027F9C2E7216B51B10C
:10EB400004F14003994204D0284600F043FAB4F996
:10EB50000C200023236300232069636022F0240239
:10EB60002060C5E742F0400209232B604FF0FF30E0
:10EB7000A28138BD08020020024B13B1024800F008
:10EB800005B8704700000000F9ED40000023014681
:10EB90001A46184600F0DABFB1F90C309AB22DE9E6
:10EBA000F0410D46110780463AD46A6843F4006389
:10EBB000002AAB816FDDAC6A002C49D000229BB2E9
:10EBC000D8F80060C8F8002013F4805267D02A6D8E
:10EBD0005F0705D569682B6B521A0BB1EB6BD21A24
:10EBE0000023E9694046A047441C3CD0B5F90C30ED
:10EBF0002A692A6023F400630022AB81DB046A6087
:10EC000047D4296BC8F8006011B305F1400399425D
:10EC100002D0404600F0DEF900202863BDE8F08114
:10EC20002E69AEB12C682E6091070CBF6B69002372
:10EC3000A41BAB600AE0234632466F6AE96940468E
:10EC4000B8470028A4EB0004064404DD002CF2DCE5
:10EC50000020BDE8F081AB8943F04003AB814FF069
:10EC6000FF30BDE8F081D8F800401D2CF3D8194BD7
:10EC7000E340DB4313F00103EDD1B5F90C206B60E9
:10EC800022F400632969AB81DA042960B9D5002C2C
:10EC9000B7D12865B5E7EA6B002A8CDCD8E70123F9
:10ECA000E9694046A047431C024602D0AB89AC6AE2
:10ECB0008EE7D8F80030002BF8D01D2B01D0162B92
:10ECC00002D1C8F80060C3E7AB8943F04003AB81D1
:10ECD000BDE8F0810100402038B50D46044608B17A
:10ECE000836BBBB1B5F90C0088B16B6EDB0701D447
:10ECF000810517D520462946FFF74EFF6B6EDA07D0
:10ED0000044602D4AB899B0507D5204638BD04468E
:10ED1000204638BD00F038F8E4E7A86D00F0F6FBB7
:10ED2000204638BDA86D00F0EFFBE3E7014900F095
:10ED3000AFBB00BF35FC400010B500230446818105
:10ED4000C281036043608360436603614361836102
:10ED5000194608225C30FEF719FE07480749084AA1
:10ED6000084B2062E4616162A262E36204F1580030
:10ED7000BDE8104000F0C4BB79F940009DF94000A7
:10ED8000D9F94000F9F9400010B50446124800F0E6
:10ED9000BBFBA26BD2B904F53B731048C4F8E83250
:10EDA0000321C4F8E022E063C4F8E412606804219F
:10EDB000FFF7C2FF01220921A068FFF7BDFF022271
:10EDC0001221E068FFF7B8FF0123A3630248BDE802
:10EDD000104000F09BBB00BF981B00202DED4000B1
:10EDE000014800F091BB00BFAC1B0020014800F0BF
:10EDF0008DBB00BFAC1B002038B50A4C0A4D641B0C
:10EE0000A4100AD004F18043013B05EB8305013CCB
:10EE100055F804399847002CF9D1BDE8384001F085
:10EE20002BBC00BF88064100840641002DE9F04755
:10EE300082B080468946144600F054FB012836D043
:10EE40004A4604F15C0301A9404600F031FE421C31
:10EE5000064625D0A8B39DF804E000250DF1040A6C
:10EE600009E023685A1C226083F800E00135B542AE
:10EE700027D215F80AE0A368013B002BA360F0DA63
:10EE8000A769BB4271462246404602DBBEF10A0F2B
:10EE9000E7D100F0B5FD431CE8D102B0BDE8F08732
:10EEA000A38943F04003A38102B0BDE8F08709F1D4
:10EEB000FF33FE2BC4D85FFA89FE06468DF804E0C6
:10EEC000CBE7484602B0BDE8F08700BF30B5536ECF
:10EED00013F0010FB2F90C30144683B005469AB214
:10EEE00001D190051CD5900406D4626E43F4005302
:10EEF00042F40052A381626628462246FFF796FF3D
:10EF0000636EDA07054602D4A3899B0502D528461D
:10EF100003B030BDA06D00F0F9FA284603B030BD53
:10EF2000A06D019100F0F0FAB4F90C3001999AB299
:10EF3000D9E700BFF8B5244F0C460646FEF774FD2E
:10EF4000BB685D68C4F57E610F3125F00305294477
:10EF500021F47F6121F00F01A1F58054B4F5805FA9
:10EF600007DB00213046FEF76BFDBB682B4498425F
:10EF700004D03046FEF75EFD0020F8BD6142304609
:10EF8000FEF75EFD01300DD0104BBA6819682D1BDD
:10EF900045F001053046091B55601960FEF74AFD32
:10EFA0000120F8BD00213046FEF74AFDBA68831AF9
:10EFB0000F2BDEDD064C0549246843F00103001BDE
:10EFC00053600860D5E700BF38060020900E00208F
:10EFD000400A0020002944D02DE9F0410D4680462A
:10EFE000FEF722FD55F8047C694927F00103A5F1DD
:10EFF0000804E2188E685068B24220F003005ED028
:10F00000FE0750600BD455F8087CE41B01F1080E94
:10F01000A56875453B446DD0E768EF60BD60151885
:10F020006D68ED073ED543F001026260E350B3F531
:10F03000007F17D2DB08581C9A104D6851F83070C9
:10F04000A7600123934001EBC0022B43083AE26022
:10F050004B6041F83040FC604046BDE8F041FEF7AF
:10F06000E9BC70475A0A042A52D89A0902F13907B2
:10F07000FF0002F13805C819CA59083890424FD02C
:10F08000516821F003018B4232D292689042F7D14D
:10F09000C368A060E3609C60C4604046BDE8F04186
:10F0A000FEF7C8BC95683B4FBD42034440D0D068D2
:10F0B000E86043F0010285606260E350B7E7FF0754
:10F0C000034407D455F8082CA41A1344A068E26836
:10F0D000C2609060304A126843F001009342606061
:10F0E0008C60B9D32D4B40461968FFF723FFB3E777
:10F0F0001046CDE711184968C90744D49168D26811
:10F10000CA60034443F0010091606060E350A3E7EC
:10F11000142A16D802F15C07FF0002F15B05AAE78A
:10F12000AA1001234D6893402B434B600346B0E780
:10F1300043F001024C610C61E560A5606260E35040
:10F140008AE7542A06D81A0B02F16F07FF0002F172
:10F150006E0590E7B2F5AA7F06D8DA0B02F17807C0
:10F16000FF0002F1770586E740F25450824206D84C
:10F170009A0C02F17D07FF0002F17C057BE74FF45A
:10F180007E777E2577E743F001016160136063E7D6
:10F190003806002040060020440A0020C00E00204F
:10F1A0009368002B73D02DE9F04F8B8983B00C4608
:10F1B00019070090164626D5226922B313F00200E3
:10F1C00035682CD04FF00009B04FC846B246B8455C
:10F1D00043464A4628BF3B460098B8F1000F50D03E
:10F1E000E169666AB047002858DDDAF808301B1A72
:10F1F0008144A8EB0008CAF80830002BE7D10020B2
:10F2000003B0BDE8F08F21460098FFF751FC0028BD
:10F2100040F03381A389356813F00200D2D113F096
:10F22000010945D14F46019637B39A05D4F80880B5
:10F2300040F183804745C346C0F0AB8013F4906F24
:10F2400040F0AC802068BA465A464946FEF73AFB81
:10F25000A2682368A2EB08025B44A2602360019AC3
:10F260009368A3EB0A03D144A7EB0A079360002B32
:10F27000C5D0A389002FD8D1D5F800906F68083584
:10F28000D2E7D5F80090D5F8048008359FE7002034
:10F29000704721460098FFF71FFD70B3B4F90C309A
:10F2A00043F040034FF0FF30A38103B0BDE8F08F7F
:10F2B000814633464E46A8469A464D464EB380B3E5
:10F2C000206823696269B145CB4628BFB34698429E
:10F2D0005F4604D9A36813449B4500F3A680934579
:10F2E0004BDB1346676AE16900982A46B847071E58
:10F2F000D4DDB9EB0709CCD00120DAF80830DB1BEC
:10F300003D44F61BCAF80830002B3FF478AF002EBE
:10F31000D5D108F1080313E9600098460833002EA0
:10F32000F9D032460A212846FEF7E2F9002800F01B
:10F33000A1800130A0EB0509C2E72068236998424B
:10F3400002D863699F425DD2B84528BFB84642469D
:10F350004946FEF7B7FAA3682268A3EB08034244C4
:10F36000A36022600BB1C24679E721460098FFF7FF
:10F37000B3FC002892D1C24671E75A462946FEF7EF
:10F38000A1FAA2682368A2EB0B025B44A26023608F
:10F39000AFE72068B846BA46BB4655E762692068C1
:10F3A000216902EB4208A0EB010A08EBD8780AF1C8
:10F3B00001004FEA680838444045424684BF804611
:10F3C00042465B0544D511460098FDF7DBFE8346B7
:10F3D000002855D052462169FEF7DAF9A38923F4B3
:10F3E000906343F08003A3810BEB0A00A8EB0A03B0
:10F3F000C4F810B0C4F814802060A360B846BA46C0
:10F40000BB4621E76FF00041B94228BF39464A4662
:10F4100091FBF3F10098666A03FB01F3E169B047E1
:10F42000B0F1000A3FF71BAF38E71A4629460193AF
:10F43000FEF748FA2268019B00981A442260214690
:10F44000FFF74AFC019B00287FF428AF1F4650E7D6
:10F45000009800F0EBF883460028C5D1009D216993
:10F460002846FFF7B7FDB4F90C300C2223F08003D7
:10F470002A6015E706F1010922E74FF0FF30BFE6E9
:10F48000009A0C231360B4F90C3009E700FCFF7FED
:10F490002DE9F84310F538771FD0884606464FF01F
:10F4A00000097D68BC68013D11D4A389012B05F1D9
:10F4B000FF3508D9B4F90E3001332146304602D069
:10F4C000C04749EA00096B1C04F16804EDD13F68AC
:10F4D000002FE6D14846BDE8F883B9464846BDE866
:10F4E000F88300BF044B054A1B685B6B002B08BF09
:10F4F000134693F828017047080200204C0A0020A8
:10F50000704700BF704700BF704700BF704700BF23
:10F5100070B50C46B1F90E10002990B015461E4684
:10F5200014DB01AA00F0E8FB00280FDB029A02F4CA
:10F530007042A2F50052B2FA82F252094FF480638F
:10F540004FF4006032602B6010B070BDA2890023C0
:10F5500012F08000336004D0402218462A6010B0B8
:10F5600070BD4FF480632B6010B070BD8A89920724
:10F570000B4606D501F1430201211A601A61596157
:10F580007047F0B583B001AB6A460C460646FFF7FC
:10F59000BFFF009905463046FDF7F4FDB4F90C3085
:10F5A000D8B1019A154F0099F76343F08003A38106
:10F5B0002060206161611AB92B43A38103B0F0BDC3
:10F5C0003046B4F90E1000F0ABFBA0B1A38923F0D4
:10F5D000030343F001031BB2EEE79A05EED423F0D8
:10F5E000030304F1430243F002030121A3812260DB
:10F5F00022616161E2E7B4F90C30DDE72DED4000F6
:10F6000082B049B15AB16BB113780B601278101CFB
:10F6100018BF012002B0704701A9002AF3D110469B
:10F6200002B070476FF00100F4E700BF002900F05E
:10F6300095802DE9F04F0D46164683B0804606F1C1
:10F640000B07FEF7F1F955F804EC162F2EF0030422
:10F65000A5F108093CD810221746BE423DD8944275
:10F6600043DAC44B996809EB0400884200F0B48087
:10F67000436823F0010101444968C9074CD51EF0D5
:10F68000010F00F09B8031464046FDF77BFD0646AA
:10F6900000283AD055F8043C23F001034B44A0F174
:10F6A00008029A4200F02181221F242A00F20781D9
:10F6B000132A00F2DB8003462A461168196051685C
:10F6C000596092689A6029464046FFF783FC1CE027
:10F6D00027F00707002F3A46BFDA00260C233046F2
:10F6E000C8F8003003B0BDE8F08F2E46E31B0F2BA7
:10F6F0001ED8D9F8043003F0010323434C44C9F861
:10F700000430636843F0010363604046FEF792F9FA
:10F71000304603B0BDE8F08F23F00303E1189142B7
:10F720001FDBC36882682E46D3600C469A60DDE713
:10F73000D9F8042009EB070102F001024C4443F020
:10F7400001031743C9F804704B60636843F0010379
:10F75000083163604046FFF73DFCD6E71146FDF7F0
:10F7600011BD1EF0010F8ED155F8081CA9EB010A3E
:10F77000DAF8041021F003010B442344934225DB03
:10F78000C26881685646CA609160DAF80C1056F873
:10F79000080F221F242AC160886000F29480132A77
:10F7A0006FD92968CAF808106968CAF80C101B2AB2
:10F7B00000F2A28008350AF1100263E055F8083C17
:10F7C000A9EB030ADAF8041021F00301631893424D
:10F7D000FFF659AF5646D8E7416821F0030BA34422
:10F7E00007F11000834556DA1EF0010F7FF44BAF8E
:10F7F00055F8081CA9EB010ADAF8041021F00301FE
:10F800008B445845E2DC5646DAF80C1056F8080FDF
:10F81000221F242AC160886000F28F80132A40F2E0
:10F820008A802968CAF808106968CAF80C101B2A6F
:10F8300000F28A8008350AF11002296811606968AF
:10F840005160A96891600AEB0701ABEB070242F037
:10F85000010299604A60DAF8043003F001031F43A3
:10F860004046CAF80470FEF7E5F851E72B680360DC
:10F870006B6843601B2A2DD800F1080305F10802CC
:10F880001BE732462968116069685160A968916078
:10F890001C46D1462AE709EB0701ABEB070B4BF0FF
:10F8A000010299604A6055F8043C03F001031F43CC
:10F8B000404645F8047CFEF7BDF82E4628E7294669
:10F8C000FEF700F8FFE6294630461C46D146FDF714
:10F8D000F9FF0BE7AB688360EB68C360242A17D09D
:10F8E00000F1100305F11002E7E650F8043C23F0A4
:10F8F00003031C442E46F9E6A968CAF81010E9680B
:10F90000CAF81410242A0CD010350AF11802B9E7ED
:10F910002B6903616B69436105F1180200F118035B
:10F92000CBE62A69CAF818206A69CAF81C2018357B
:10F930000AF12002A6E732467FE7294630460193C6
:10F94000FDF7C0FF019B7EE7A968CAF81010E968BF
:10F95000CAF81410242A03D010350AF118026CE7F3
:10F960002A69CAF818206A69CAF81C2018350AF1F1
:10F97000200262E73806002010B50C46B1F90E10DF
:10F9800000F0F6F9002803DB236D0344236510BD66
:10F99000A38923F48053A38110BD00BF2DE9F0415A
:10F9A0001646B1F90C201F46D3050C46054607D56F
:10F9B00000220223B1F90E1000F0C4F9B4F90C20B2
:10F9C000B4F90E1022F48052A2813B4632462846FA
:10F9D000BDE8F04100F0A4B810B50C46B1F90E1026
:10F9E00000F0B0F9A389421C0EBF23F4805343F406
:10F9F00080532065A38110BDB1F90E1000F008B945
:10FA0000F8B50D461446064610B1836B002B4BD05B
:10FA1000B4F90C20A369A36091B2080739D5236912
:10FA2000002B36D0EDB289042F4615D522686169C6
:10FA3000D31A8B421CDA0133A168501C0139A16032
:10FA40002060157062699A421AD0A389DB0701D53C
:10FA50000A2D15D03846F8BD616E42F4005221F4EB
:10FA60000051A281226861666169D31A8B42E2DB90
:10FA700021463046FFF730F940B922680123DBE721
:10FA800021463046FFF728F90028E3D04FF0FF3732
:10FA9000E0E721463046FFF70BF80028F6D1B4F92D
:10FAA0000C20236991B2BDE7FFF76EF9B0E700BF04
:10FAB000F0B5064685B01F4689B1104C104D24683C
:10FAC000646B002C08BF2C46D4F8E040A047431CD0
:10FAD00003D100228A233A60336005B0F0BD0C46A2
:10FAE0000649074A0968496B002908BF11462246A2
:10FAF000D1F8E04001A9A047E9E700BF08020020D3
:10FB00004C0A002021B1FF2A04D80A700120704756
:10FB1000084670478A2303604FF0FF30704700BFEC
:10FB200070B50D46084C114606461A462846002375
:10FB30002360FAF727FB431C00D070BD2368002B1D
:10FB4000FBD0336070BD00BFB01B00202DE9F8432F
:10FB50002C4D0646286898460F469146FFF7D4FC80
:10FB6000294B1C68D4F84831002B3ED05A681F2A14
:10FB70001CDC02F1010E76B103EB82010124C1F815
:10FB80008890D3F8880194402043022EC3F888015E
:10FB9000C1F8088123D00232C3F804E0286843F892
:10FBA0002270FFF7B3FC0020BDE8F883174B0BB3BE
:10FBB0004FF4C870FDF7D6FA0346D8B1D4F84821FF
:10FBC0000260002141600A46C4F848014FF0010E6E
:10FBD000C0F88811C0F88C11002EDCD0CCE7D3F827
:10FBE0008C110C43C3F88C41D5E704F5A673C4F817
:10FBF0004831BBE72868FFF789FC4FF0FF30BDE8CC
:10FC0000F88300BF480A0020FC04410065D1400091
:10FC100038B5074C0023054608462360FAF7B4FEC2
:10FC2000431C00D038BD2368002BFBD02B6038BDAF
:10FC3000B01B002070B559B105460C4610B1836B5E
:10FC4000002B3CD0636ED80705D5B4F90C302BB926
:10FC50000026304670BDA38999053CD5214628462B
:10FC6000FEF79AFFE36A064633B1E16928469847F2
:10FC70000028B8BF4FF0FF36A3891A0622D4216BA3
:10FC800041B104F14003994202D02846FFF7A2F99E
:10FC900000232363616C21B12846FFF79BF9002301
:10FCA0006364FFF79DF8636E0022DB07A2810ED527
:10FCB000A06DFFF727FCFFF799F8304670BDFFF7FE
:10FCC00063F8BFE721692846FFF784F9D7E7A06DFD
:10FCD000FFF71CFCECE7A06DFFF716FCB4F90C3045
:10FCE000002BBBD1666E16F00106B1D1A06DFFF7F7
:10FCF0000DFC304670BD00BF38B50B46074C0546BD
:10FD00001146184600232360FAF741FE431C00D039
:10FD100038BD2368002BFBD02B6038BDB01B002002
:10FD200038B5074C0023054608462360FAF734FE31
:10FD3000431C00D038BD2368002BFBD02B6038BD9E
:10FD4000B01B002070B50D46084C114606461A46F9
:10FD5000284600232360FAF721FE431C00D070BD23
:10FD60002368002BFBD0336070BD00BFB01B0020A8
:10FD700070B50D46084C114606461A462846002323
:10FD80002360FAF7E5F9431C00D070BD2368002B0F
:10FD9000FBD0336070BD00BFB01B002053B94AB91F
:10FDA000002908BF00281CBF4FF0FF314FF0FF3083
:10FDB00000F07AB9ADF1080C6DE904CE00F006F858
:10FDC000DDF804E0DDE9022304B070472DE9F047D7
:10FDD0008C460D460446089E002B51D18A42174698
:10FDE0006DD9B2FA82FEBEF1000F0BD0CEF1200C1D
:10FDF00001FA0EF520FA0CFC02FA0EF74CEA050C9B
:10FE000000FA0EF44FEA174A250CBCFBFAF81FFA69
:10FE100087F90AFB18CC45EA0C4508FB09F3AB420D
:10FE20000AD9ED1908F1FF3280F02381AB4240F28C
:10FE30002081A8F102083D44ED1AA4B2B5FBFAF006
:10FE40000AFB105544EA054400FB09F9A14509D90C
:10FE5000E41900F1FF3380F00A81A14540F20781E7
:10FE600002383C44A4EB090440EA08400021002E7B
:10FE700061D024FA0EF4002334607360BDE8F0878B
:10FE80008B4207D9002E54D0002186E82100084675
:10FE9000BDE8F087B3FA83F1002940F08E80AB42D1
:10FEA00002D3824200F2FA80841A65EB0305012036
:10FEB000AC46002E3FD086E81010BDE8F08712B99E
:10FEC0000127B7FBF2F7B7FA87FEBEF1000F34D176
:10FED000EB1B3A0C1FFA87FC0121B3FBF2F8250C4F
:10FEE00002FB183345EA03450CFB08F3AB4207D984
:10FEF000ED1908F1FF3002D2AB4200F2D18080460A
:10FF0000ED1AA3B2B5FBF2F002FB105543EA05442B
:10FF10000CFB00FCA44507D9E41900F1FF3302D221
:10FF2000A44500F2B8801846A4EB0C0440EA08404F
:10FF30009DE731463046BDE8F087CEF1200405FA52
:10FF40000EF307FA0EF720FA04F83A0C25FA04F437
:10FF500048EA0308B4FBF2F14FEA184502FB1144EA
:10FF60001FFA87FC45EA044501FB0CF3AB4200FA9B
:10FF70000EF409D9ED1901F1FF3080F08A80AB420F
:10FF800040F2878002393D44EB1A1FFA88F5B3FB33
:10FF9000F2F002FB103345EA034500FB0CF3AB42E1
:10FFA00007D9ED1900F1FF386FD2AB426DD9023895
:10FFB0003D44EB1A40EA01418FE7C1F1200722FAE4
:10FFC00007F88B4005FA01F448EA030320FA07FE1C
:10FFD0004FEA134CFD404EEA040EB5FBFCF94FEA24
:10FFE0001E440CFB19551FFA83F844EA054509FB2A
:10FFF00008F4AC4202FA01F200FA01FA08D9ED184D
:020000040041B9
:1000000009F1FF3043D2AC4241D9A9F102091D44A4
:100010002D1B1FFA8EFEB5FBFCF00CFB10554EEAB3
:10002000054400FB08F8A04507D9E41800F1FF35A6
:1000300029D2A04527D902381C4440EA0940A4EB44
:100040000804A0FB02894C45C6464D4615D312D084
:1000500056B1BAEB0E0364EB050404FA07F7CB4084
:100060001F43CC40376074600021BDE8F08718461C
:10007000F8E69046E0E6C245EAD2B8EB020E69EB3C
:1000800003050138E4E72846D7E7404691E7814673
:10009000BEE7014678E702383C4445E7084608E7F2
:1000A000A8F102083D442BE7704700BF01000000A3
:1000B0000200000004000000080000001000000022
:1000C00020000000400000008000000000008000D0
:1000D0000000000100000002000000040000000811
:1000E0000000001000000000000000000000000000
:1000F0000000000000000000000000000000000000
:1001000000000000000000000000000001280110B5
:100110000253290351FF01026902026B100580019D
:1001200040401103F0AA1104C00040000AC2010AB5
:10013000010A010A0090022D701100008910800749
:100140008003C0078003C003C0020003580020C61C
:1001500037000D000F00110008180010F0030C20EC
:1001600000060B0B3308810256000B0011000882B9
:100170000256000B00110002350002250103F0AA0F
:100180001002D10203F0AA110AC2010A010A010AEF
:1001900000900203FF5A8102650B0EF9585F666DED
:1001A000747B828990979EA5AC03F0AA1202D3209B
:1001B00003BF37BE02038102360003F0AA1104C553
:1001C000000140000128011002038102532903515C
:1001D000FF01026900026B102D7011000089108070
:1001E00009F004F804F804F804F80200041B0020E5
:1001F00091BF0011000F00190009180010F0030C46
:100200002000060B0B330580013E3E11088101E101
:100210000010001000088201E1001000100002250B
:100220000103F0AA1002D10203F0AA110AC2010AC6
:10023000010A010A00900203F0AA1202D32003BFB0
:1002400007BE03FF5A8102650B0EF9585F666D7495
:100250007B828990979EA5AC00000000FF00FF0004
:10026000565852303000000055534152540000009F
:100270004661696C656420746F20637265617465A2
:10028000207573617274207461736B0D0A00000035
:1002900000FFFFFFFFFFFF0009273412D204000018
:1002A000021E0104A5000078E70000000000000025
:1002B0000000000000000101010101010101010134
:1002C0000101010101010000000000000000000028
:1002D0000000FFFF00000018000000000000000008
:1002E000000000000000000000000000000000000E
:1002F000000000000000000000000000000000FC02
:10030000004265796F6E6400000000000000010D7E
:10031000702079000022092839540F80DF137F00F4
:100320003F801F00EF0917000E8001001EF50A0034
:10033000FF0EFF003F801F007F071B000E800100A3
:100340007E00073A029281000800000000000000D1
:10035000000000000000000000000000000000009D
:10036000000000000000000000000000000000008D
:10037000000000000000000000000000000000007D
:100380000000000000000000000000000000F890E5
:100390005265706F727400004661696C6564207408
:1003A0006F206372656174652048494420726570EE
:1003B0006F7274207461736B0D0A00004932430040
:1003C0004661696C656420746F2063726561746551
:1003D00020493243207461736B0D0A0054494D4526
:1003E000445F5354415254004661696C6564207403
:1003F0006F206372656174652074696D6564207334
:10040000746172747570207461736B0D0A00000062
:10041000414443004661696C656420746F206372D7
:100420006561746520414443207461736B0D0A005B
:1004300049444C450000000000C20100C00000001B
:1004400000080000000000002D2D20467265657236
:10045000746F73204578616D706C65202D2D0A0DC9
:1004600000000000444953504C4159424F4152440E
:100470002056302E342E31002D2D2025730A0D00EC
:1004800031323A33323A3235000000004F63742083
:1004900020372032303232002D2D20436F6D7069AD
:1004A0006C65643A202573202573202D2D0A0D00DC
:1004B0005553424C6F6164004661696C65642074F9
:1004C0006F2063726561746520555342204C6F61E3
:1004D000646572207461736B0D0A0000737461634C
:1004E0006B206F766572666C6F7720257820257398
:1004F0000D0A00006C6F676600000000100200200B
:100500003031323334353637383941424344454649
:10051000000000003031323334353637383961620B
:100520006364656600000000286E756C6C2900002D
:1005300020202020202020202020202020202020BB
:1005400030303030303030303030303030303030AB
:1005500043000000504F5349580000002E00000097
:100560000020202020202020202028282828282083
:10057000202020202020202020202020202020207B
:1005800020881010101010101010101010101010E3
:1005900010040404040404040404041010101010D3
:1005A000101041414141414101010101010101019D
:1005B00001010101010101010101010110101010EF
:1005C000101042424242424202020202020202026F
:1005D00002020202020202020202020210101010C3
:1005E00020000000000000000000000000000000EB
:1005F00000000000000000000000000000000000FB
:1006000000000000000000000000000000000000EA
:1006100000000000000000000000000000000000DA
:1006200000000000000000000000000000000000CA
:1006300000000000000000000000000000000000BA
:1006400000000000000000000000000000000000AA
:10065000000000000000000000000000000000009A
:1006600000000000F8B500BFF8BC08BC9E4670470B
:1006700079EB400029444000F8B500BFF8BC08BC45
:100680009E4670470544400044F7FF7F010000008C
:1006900030B482B0049C5BB31D46036843F48033DE
:1006A0000360C9B241F0B441416083680193019B8A
:1006B00013F0010FF9D1002306E0990001F5800144
:1006C000096845F823100133A342F6D3D2B242F0B1
:1006D000B442426083680193019B13F0010FF9D08B
:1006E000036823F480330360002002B030BC7047FD
:1006F0000220FAE70160704782B04160836801938D
:10070000019B13F0010FF9D0019800F00E0002B028
:100710007047FFFFFFFF0000994540009D454000E6
:100720009F454000A3454000A7454000E1454000EB
:1007300031464000A9454000AD454000B945400064
:100740000147470150010020C000002000000000C8
:10075000C80000206401002009028500030100C0D8
:1007600032080B000201010002090400000001012F
:10077000000209240100011E0001010C24020101F4
:10078000020002030000000924030201010001002D
:100790000904010000010200020904010101010233
:1007A0000002072401020101000B240201020210D1
:1007B0000180BB0009058405000101000007250137
:1007C00000000000090402000103000000092111DB
:1007D00001000122260007058103400004000000FB
:1007E0001201000200000040BD35010100010102BC
:1007F00000010000880000209C0000207001002003
:1008000089754000A975400001764000AB75400035
:100810000000000006FFFF0901A1010902090315FC
:100820000026FF007508954081020906090715009A
:1008300026FF0075089540B102C0000000030000CB
:1008400000000000000000000000000000000000A8
:100850000000000000000000000000000000000098
:1008600000000000000000000403090447656E65F5
:10087000726963005553422053746572656F204D51
:100880006963726F70686F6E6500010000127A0014
:10089000AAAAAAAA0100000010020020000000007D
:1008A00000000000FC04002064050020CC050020AE
:1008B0000000000000000000000000000000000038
:1008C0000000000000000000000000000000000028
:1008D0000000000000000000000000000000000018
:1008E0000000000000000000000000000000000008
:1008F00000000000000000000000000000000000F8
:1009000000000000000000000000000000000000E7
:1009100000000000000000000000000000000000D7
:1009200000000000000000000000000000000000C7
:1009300000000000000000000000000000000000B7
:1009400000000000000000000100000000000000A6
:100950000E33CDAB34126DE6ECDE05000B0000006B
:100960000000000000000000000000000000000087
:100970000000000000000000000000000000000077
:100980000000000000000000000000000000000067
:100990000000000000000000000000000000000057
:100CD000380600203806002040060020400600208C
:100CE000480600204806002050060020500600203C
:100CF00058060020580600206006002060060020EC
:100D0000680600206806002070060020700600209B
:100D1000780600207806002080060020800600204B
:100D200088060020880600209006002090060020FB
:100D30009806002098060020A0060020A0060020AB
:100D4000A8060020A8060020B0060020B00600205B
:100D5000B8060020B8060020C0060020C00600200B
:100D6000C8060020C8060020D0060020D0060020BB
:100D7000D8060020D8060020E0060020E00600206B
:100D8000E8060020E8060020F0060020F00600201B
:100D9000F8060020F80600200007002000070020C9
:100DA0000807002008070020100700201007002077
:100DB0001807002018070020200700202007002027
:100DC00028070020280700203007002030070020D7
:100DD0003807002038070020400700204007002087
:100DE0004807002048070020500700205007002037
:100DF00058070020580700206007002060070020E7
:100E00006807002068070020700700207007002096
:100E10007807002078070020800700208007002046
:100E200088070020880700209007002090070020F6
:100E30009807002098070020A0070020A0070020A6
:100E4000A8070020A8070020B0070020B007002056
:100E5000B8070020B8070020C0070020C007002006
:100E6000C8070020C8070020D0070020D0070020B6
:100E7000D8070020D8070020E0070020E007002066
:100E8000E8070020E8070020F0070020F007002016
:100E9000F8070020F80700200008002000080020C4
:100EA0000808002008080020100800201008002072
:100EB0001808002018080020200800202008002022
:100EC00028080020280800203008002030080020D2
:100ED0003808002038080020400800204008002082
:100EE0004808002048080020500800205008002032
:100EF00058080020580800206008002060080020E2
:100F00006808002068080020700800207008002091
:100F10007808002078080020800800208008002041
:100F200088080020880800209008002090080020F1
:100F30009808002098080020A0080020A0080020A1
:100F4000A8080020A8080020B0080020B008002051
:100F5000B8080020B8080020C0080020C008002001
:100F6000C8080020C8080020D0080020D0080020B1
:100F7000D8080020D8080020E0080020E008002061
:100F8000E8080020E8080020F0080020F008002011
:100F9000F8080020F80800200009002000090020BF
:100FA000080900200809002010090020100900206D
:100FB000180900201809002020090020200900201D
:100FC00028090020280900203009002030090020CD
:100FD000380900203809002040090020400900207D
:100FE000480900204809002050090020500900202D
:100FF00058090020580900206009002060090020DD
:10100000680900206809002070090020700900208C
:10101000780900207809002080090020800900203C
:1010200088090020880900209009002090090020EC
:101030009809002098090020A0090020A00900209C
:10104000A8090020A8090020B0090020B00900204C
:10105000B8090020B8090020C0090020C0090020FC
:10106000C8090020C8090020D0090020D0090020AC
:10107000D8090020D8090020E0090020E00900205C
:10108000E8090020E8090020F0090020F00900200C
:10109000F8090020F8090020000A0020000A0020BA
:1010A000080A0020080A0020100A0020100A002068
:1010B000180A0020180A0020200A0020200A002018
:1010C000280A0020280A0020300A0020300A0020C8
:1010D000FFFFFFFF000002008C1B00204300000008
:1010E0000000000000000000000000000000000000
:1010F00000000000000000000000000043000000AD
:1011000000000000000000000000000000000000DF
:10111000000000000000000000000000430000008C
:1011200000000000000000000000000000000000BF
:10113000000000000000000000000000430000006C
:10114000000000000000000000000000000000009F
:10115000000000000000000000000000430000004C
:10116000000000000000000000000000000000007F
:10117000000000000000000000000000430000002C
:10118000000000000000000000000000000000005F
:10119000000000000000000000000000430000000C
:1011A000000000000000000000000000000000003F
:1011B00000000000000000000000000005FB4000EF
:1011C00001F6400000000000600541005C054100A0
:1011D000600441006004410060044100600441007B
:1011E000600441006004410060044100600441006B
:1011F00060044100FFFFFFFFFFFFFFFFFFFFFFFF56
:10120000FFFF000001004153434949000000000076
:1012100000000000000000000000000000000000CE
:101220000000000000004153434949000000000055
:1012300000000000000000000000000000000000AE
:101240000000000000000000FFFFFFFFFFFFFFFFA6
:10125000FFFFFFFFFFFFFFFFFFFFFFFF150453D15D
:00000001FF
